:020000040000FA
:1000000004000400C5EF0FF0086A800E3A6E39D084
:10001000196A1A6A0A9A5BEC02F0D8A01200D30F90
:10002000D8B40A8A2D0FC60F03E20A0FF4E305D0F5
:10003000F30FF1E2060FEFE30A0F156E040E166ED2
:10004000D89019361A36162EFBD7155019120806F5
:100050000FE05BEC02F0D8A01200C60F03E20A0F1B
:1000600007E3EBD7F30F04E2060F02E30A0FE5D72D
:100070000AAA04D0191E1A1E194A1A2A1950D88021
:100080001200196A1A6A1B6A1C6A0A9A5BEC02F06F
:10009000D8A01200D30FD8B40A8A2D0FC60FF6E2EB
:1000A0000A0FF4E3156E146A136A126A0A0E116ECF
:1000B00029EC04F015501124196E12501A6E000E1E
:1000C000D8B0010E1A2613501B6E000ED8B0010EC8
:1000D0001B2614501C6E000ED8B0010E1C260806FC
:1000E00007E0E9D9D8A01200C60F02E20A0FDAE24F
:1000F0000AAA0BD0191E1A1E1B1E1C1E192AD8B4C0
:100100001A2AD8B41B2AD8B41C2A1950D880120035
:10011000086A196E1A6A00960850D8B40086040E50
:10012000076E1A3805D81A5003D8193801D8195053
:100130000F0BF60FD8B0070F0A0F23D032D803D019
:10014000086A196E1A6A00960850D8B40086050E1F
:10015000076E270E166E100E0CD8030E166EE80EE4
:1001600008D8166A640E05D8166A0A0E02D8195005
:1001700008D0156E1A50126E1950116ED7EC03F09C
:100180001150116E074E0096085003E0075CD8B07E
:1001900007D01150D8A4009600B602D0300F7BD102
:1001A00012001AAE120019501A10D8B41200191EFB
:1001B0001A1E194A1A2A2D0E6ED13C6E25AE02D097
:1001C0002D0E69D9273E04D0263E02D0254A252A85
:1001D000326A336A346A356A258E6A0E2426D890CC
:1001E0002532263227323532343233323232243E0F
:1001F000F6D72750245C2726245E2650255C262629
:10020000255E086A38D82E0E46D93D6AD890323419
:10021000276E3334266E3434256E3534246E3D36E5
:10022000D89027362636253624363D3632502726B6
:100230003350D8B0333C26263450D8B0343C252631
:100240003550D8B0353C2426D8B03D3ED89027361E
:100250002636253624363D363D50300F1CD927C072
:1002600032F026C033F025C034F024C035F03C2EE7
:10027000CCD7D89012000096085003E100860A0EF1
:10028000086E27C014F026C013F025C012F024C059
:1002900011F0076A1C6A1B6A1A6A0A0E196EA9EC29
:1002A00003F0072A0750085CD8A4F4D71950D8A443
:1002B000009600A602D0082C03D01950300FEBD8BE
:1002C000082EDFD7120005C011F006C012F0010E93
:1002D000156E166AEA6802C0E9FF04002BD8D8A0A0
:1002E00016D0152EFAD7FF0E1626D8B0F6D711263F
:1002F000D8A01226D8A01200200E156E030E166E7E
:10030000ECD7EA6802C0E9FF040014D8FDE254D833
:100310001F6A080E166E51D80DD8D8B01F3E153280
:10032000162EF9D722AA1F6A22BA159E46D8D8805F
:1003300015501200120EE9260950EF1202C0E9FF13
:10034000EF1422BC0918FF0F12001D6EEA68E26864
:100350000250E96E120FE16E800E0A16080E1E6E34
:10036000D890D8B00A3E11D81D321E2EFAD70400FC
:1003700022BA0A300AD800D000D000D0D88005D8E0
:100380000650166E05509FD9120022AE0BD0EF50CA
:10039000091022AC0918EF6EE7500910D8A009180F
:1003A000E76E0BD0EF500910D8A0091822BC09182D
:1003B000EF6E091CE71601D00A8C22501F0B000FAC
:1003C000126E2150110FD8B0122A0AAC89D10A9CA2
:1003D000116E020E7BEC04F083D1ABB2AB98AB880C
:1003E00002C011F009C012F0156A166A040000D0AC
:1003F00004009EBA15D0E868152616221122122292
:10040000D8A012001548163CF1D7D00E156E030E79
:10041000166EEED7ABB2AB98AB8804009EAAFED79F
:10042000AE50D880120004009EA8FED7AD6E120018
:1004300071B27198718802C011F009C012F0156A8A
:10044000166A040000D00400A4BA15D0E868152686
:10045000162211221222D8A012001548163CF1D7FC
:10046000D00E156E030E166EEED771B271987188AC
:100470000400A4AAFED77450D8801200A66AA68EE3
:100480000900F55002E002D8FBD712000400A4A82E
:10049000FED7736E120001BA58D701B4C4D701A2B7
:1004A00002D001B03CD001A205D001B003D001B20E
:1004B000EE6E1200EBD73A5290E03A04ABE03A50BD
:1004C000080AB6E03A50090AD0E03A50030AD8B414
:1004D000FAD63A50050AD8B414D7D8803ABEEE50AE
:1004E0001200008800A8009800BA03D0008A35D80E
:1004F00029E20094080E166E40D81536162EFCD749
:1005000000B407D000B801D04AD845D841D800B8C7
:1005100019D843D8D89015501CD0008800A800984E
:1005200000BC05D0FE0B0A6E008CD89012D000BE25
:1005300005D01D6E008E11D805E21D5012D802E2C2
:1005400000A807D02CD827D8009C009E009A0094C1
:1005500024D81F80D8A01F90120017D80A5000BAC4
:100560000109156E080E166E153617D801E217D858
:1005700012D80ED8162EF8D710D80DD800D00400F7
:10058000D89081BCD88004D8120007D804D807D8E6
:10059000819E939E06D0938E04D0938C02D08A9C29
:1005A000939C1200AA6AA96EA66AA680A850A94ABE
:1005B000AA2A1200AA6AA86EA66AA684550EA76E79
:1005C000AA0EA76EA6820400A6B2FED7A694A94AD8
:1005D000AA2A1200E836E836FC0B0109C21280098B
:1005E000C216C050F80B0309C06E640E78D8C282E0
:1005F0000400C2B2FED7C4CF25F0C350246E12004F
:10060000080E1D6E1E6EEA6803C0E9FF04500AB4AE
:1006100076D90AA476D9E26803C0E1FFEA6802C08D
:10062000E9FF0950E988E92AEC1202C0E9FF116AE2
:10063000126A1D50D8B412000AB234D8EF5009140F
:10064000FF0F113612360AA22DD81D2EF5D71E50D7
:100650000AB040D111501200080E1D6EEA6803C0A6
:10066000E9FF04500AB44BD90AA44BD9E26803C08D
:10067000E1FFEA6802C0E9FF091CE988E92AEC16F3
:100680001D50D8B412000AB025D902C0E9FF1232B9
:100690001132EF500910D8A00918EF6E03D81D2EA3
:1006A000F6D712000450E71A040000D000D000D0A2
:1006B00000D000D000D000D000D000D000D000D0BA
:1006C000E71A1200166A156EFF0E1526162200D0C4
:1006D000D8A01200030E126EE60E02D8F5D7126AE9
:1006E000FE0F116E040000D000D0E86A125AD8A0A4
:1006F0001200110600D000D0F5D70009D8B41200BE
:100700001F6E11C0E9FF12C0EAFF126A116A1FBE14
:1007100007D0EE50116E1FA21200EF50126E1200A1
:1007200004D8EF14D8A4112A1200010E1FB0E84417
:100730001FB2E8441FB2E8441FB4E8381200010FAA
:100740001E6E0A0E156E166A32D81E2EFDD719506F
:1007500012002E6A2F6A306A316A210E176E15D088
:100760002E362F363036313619502E5C1A502F580F
:100770001B5030581C50315808E3316E19502E5E12
:100780001A502F5A1B50305AD88011361236133651
:100790001436172EE5D731C01CF030C01BF02FC027
:1007A0001AF02E50196E1200126A166A156E1A6A25
:1007B000196A100EF36E123419361A361550195C78
:1007C00016501A5805E31550195E16501A5AD8805B
:1007D00011361236F32EEFD71150120020501A188E
:1007E000800BF46E20AE05D01F1E201E1F2AD8B429
:1007F000202A1AAE05D0191E1A1E192AD8B41A2A90
:10080000156A116A126A166A1A5002E1195018E044
:10081000100EF36ED8901F362036153616361A5045
:10082000165C02E11950155C07E31950155ED8A05B
:1008300016061A50165ED88011361236F32EEAD7F5
:10084000F4AE05D0111E121E112AD8B4122A11506E
:10085000120014C031F013C030F012C02FF011C0DC
:100860002EF030501902F3CF13F0F4CF14F02F50C4
:100870001A02F3501326F45014222E501B02F35088
:100880001326F450142231501902F350142630501C
:100890001A02F35014262F501B02F35014262E5028
:1008A0001C02F35014262E501902F3CF11F0F4CF8E
:1008B00012F02F501902F3501226F4501322000E9A
:1008C00014222E501A02F3501226F4501322000E56
:1008D00014221200156A166A04D01232113215362B
:1008E0001636FF0FFAE216C012F01550116E120004
:1008F000D89012321132FF0FFBE211501200EF12AA
:1009000003D0FF0AEF1601D0FF0AE988E92AEC16A6
:100910001200A66AA68E0900F55002E0EE6EFBD723
:100920001200A66AA68EEE500900F55C02E1F5669B
:10093000FAD712003EC01FF03E8C0ED8D90E396E89
:100940005B0E386E5E0E376E7D0E366E6AEC07F00B
:100950001FAC3E9C3550120033BE09D13252D8B480
:1009600006D13EC01DF03E8C7E0E325C1E6E7E0EA9
:10097000326E396A386A376A7F0E366EF30E355C2E
:10098000040ED8A0050E345C350ED8A0360E335CAC
:1009900002E3AAD903D0322AA7D91E0635C011F026
:1009A00034C012F033C013F032C014F0710E396E3F
:1009B0005F0E386E550E376E800E366E97D911C0A9
:1009C00039F012C038F013C037F014C036F06AECBA
:1009D00007F0C60E396EF50E386E1F0E376E800E9C
:1009E000366E84D935C015F034C016F033C017F018
:1009F00032C018F011C035F012C034F013C033F01B
:100A000014C032F08A0E396E120E386E790E376EBF
:100A10007D0E366E6AEC07F0F60E396E460E386EB5
:100A2000550E376E7E0E366E61D915C039F016C080
:100A300038F017C037F018C036F0E6D935C015F0D9
:100A400034C016F033C017F032C018F01450326EB4
:100A5000366E1350336E376E1250346E386E11503E
:100A6000356E396E6AEC07F035C024F034C025F0DD
:100A700033C026F032C027F015C039F016C038F068
:100A800017C037F018C036F06AEC07F011C039F023
:100A900012C038F013C037F014C036F06AEC07F01B
:100AA00024C039F025C038F026C037F027C036F012
:100AB0003666360619D911C039F012C038F013C0A5
:100AC00037F014C036F012D91E5252E035C024F06F
:100AD00034C025F033C026F032C027F01EC032F0FB
:100AE000000E32BEFF0E336E346E356E17EC08F01A
:100AF00035C011F034C012F033C013F032C014F01E
:100B0000830E396E800E386EDE0E376E720E366EC4
:100B1000E1D924C039F025C038F026C037F027C00D
:100B200036F0E4D835C024F034C025F033C026F0C8
:100B300032C027F011C035F012C034F013C033F0CA
:100B400014C032F0396A800E386E310E376E7E0E68
:100B5000366EC0D924C039F025C038F026C037F031
:100B600027C036F0C3D81DBC03D03E9C01D03E8ABE
:100B70003550120037503318406E40BE30D037BE6B
:100B800017D03650325CD8A0000CD8A4010C3750D6
:100B9000335CD8A0000CD8A4010C3850345CD8A029
:100BA000000CD8A4010C3950355CD8A0000C010C05
:100BB0003250365CD8A0000CD8A4010C3350375CFE
:100BC000D8A0000CD8A4010C3450385CD8A0000C7C
:100BD000D8A4010C3550395CD8A0000C010C33AE00
:100BE000010C000C37503318406E40BE34D037BE75
:100BF00019D03650325CD8A0000CD8A4010C375064
:100C0000335CD8A0000CD8A4010C3850345CD8A0B8
:100C1000000CD8A4010C3950355CD8A0000CD8A425
:100C2000010C000C3250365CD8A0000CD8A4010C8A
:100C30003350375CD8A0000CD8A4010C3450385C79
:100C4000D8A0000CD8A4010C3550395CD8A0000CF9
:100C5000D8A4010C000C33AE010C000C3350371833
:100C6000406E40BE34D033BE19D03250365CD8A06E
:100C7000000CD8A4010C3350375CD8A0000CD8A4C9
:100C8000010C3450385CD8A0000CD8A4010C3550AD
:100C9000395CD8A0000CD8A4010C000C3650325C92
:100CA000D8A0000CD8A4010C3750335CD8A0000C9D
:100CB000D8A4010C3850345CD8A0000CD8A4010C86
:100CC0003950355CD8A0000CD8A4010C000C37AE0C
:100CD000010C000C396A386A7E0E366E800E33AE17
:100CE000000E376E03D844D1800E371A3650325C6E
:100CF0003D6E11E23D6C325036C032F0366E3350EC
:100D000037C033F0376E345038C034F0386E355059
:100D100039C035F0396E1A0E3D6074D0365272E02B
:100D20003C6A33503F6E3718416E338E378E080E53
:100D30003D5E08E339C03CF038C039F037C038F0C8
:100D4000376AF5D73D2607E0D89037323832393246
:100D50003C323D2EF9D741AE33D03950355E385054
:100D6000345A3750335A07E2D880000E355634567D
:100D70003356800E3F1A3C6C04E03506000E345AA0
:100D8000335A040E3D6E33660DD034C033F035C097
:100D900034F03CC035F03C6A080E325E29E33D2E4B
:100DA000F2D726D033BE08D0D8903C36353634360C
:100DB0003336322EF7D71CD03CAE22D03C6A0FD04F
:100DC00039503526385034223750332206E3333237
:100DD000343235323C32324A0DD03CAE11D0353E41
:100DE0000FD0343E0DD0333E0BD0D8803590EFD7A6
:100DF000326A02D03E823268356A346A800E336EBF
:100E00003FAE339E355012003350306E3718416E6E
:100E1000365051E0325252E0325E7F0E03E232260B
:100E200003E24BD032264CE235C02EF034C02FF016
:100E3000308E378E180E3F6E356A346A336A0BD0A7
:100E400039502E5C38502F5811E32F6E306A3950CC
:100E50002E5E0BD004E23750305CF2E007E33950ED
:100E60002E5E38502F5A3750305AD88035363436A7
:100E700033362E362F3630363F2EECD733BE07D0E2
:100E800032521BE0413232063F2A4136E3D707E2B5
:100E900039502E5E38502F5A3750305A17E3353EAE
:100EA00015D0343E13D0333E11D033323432353284
:100EB000323E0CD005D03E8604D03E84326A02D049
:100EC0003E823268356A346A800E336E41AE339E9C
:100ED000355012003350306E3718416E3250D8A45E
:100EE00036503AE032267E0E03E3325E03E336D01C
:100EF000325E31E335C02EF034C02FF0308E378EA5
:100F0000356A346A336A180E3F6E30322F322E3211
:100F100006E33950352638503422375033223332E5
:100F2000343235323F2EF1D733BE07D03536343622
:100F30003336325210E03206303416E3353E14D0E8
:100F4000343E12D0333E10D0D88033323432353272
:100F5000323E0AD003D03E84326A02D03E823268EA
:100F6000356A346A800E336E41AE339E35501200BE
:100F700032C03FF0335035C033F0356E35363F3236
:100F800035323E6A35363F3602E33E843E7E06E128
:100F90003E803F6A356A346A336A0BD03F2803E0EB
:100FA000D880353206D0D890353202E13E8201D069
:100FB0003E863EB604D03EA20FD03EB407D07F0E90
:100FC000356EFF0E346E336E326E23D0800E356E6A
:100FD00001D0356A000EF6D73EB0FBD7326A9F0EBD
:100FE0003F60EBD77E0E3F64F4D79E0E3F5C07E078
:100FF000D89035323432333232323F2AF6D73EA4DB
:1010000008D0D880000E325633563456355635AE99
:10101000E0D732501200000E33BEFF0E346E356E34
:1010200006D0326E336A346A356A419E0AD0419ED8
:1010300035AE07D0D880000E32563356345635566A
:10104000418E960E3F6E355209E0080E3F2633C0A2
:1010500032F034C033F035C034F011D034520FE1E7
:10106000080E3F5E335007E1080E3F5E325002E14A
:10107000355010D0326A346E32C033F0326A34BE2A
:1010800006D0D8903236333634363F06F8D741AEE4
:10109000349E3F5032C035F0326E345033C034F09D
:1010A000336E120024505542582C34302C474C4C8F
:1010B0002C302C302C302C302A3543002450554213
:1010C000582C34302C5A44412C302C302C302C30BD
:1010D0002A34340024505542582C34302C4753566F
:1010E0002C302C302C302C302A35390024505542ED
:1010F000582C34302C4753412C302C302C302C3091
:101100002A34450024505542582C34302C524D433B
:101110002C302C302C302C302A34370024505542BF
:10112000582C34302C5654472C312C302C302C3049
:101130002A35460024504D544B3331342C302C305A
:101140002C312C312C302C302C302C302C302C30BD
:101150002C302C302C302C302C302C302C302C30AF
:101160002C302A32380024504D544B3136312C303B
:101170002A32380024504D544B3130322A3331005A
:101180002447504747412C3030303030302E3030FB
:10119000302C303030302E303030302C4E2C30303F
:1011A0003030302E303030302C452C312C31302C3A
:1011B000312E322C3230302E302C4D2C2D33342E1B
:1011C000322C4D2C2C303030302A3545000024474D
:1011D000505654472C3330392E36322C542C202C78
:1011E0004D2C302E31332C4E2C302E322C4B2C41AA
:1011F0002A323300242424244E4F20454E4F554795
:101200004820534154454C49544553002424242438
:1012100047505320434F4D4D554E49434154494F3C
:101220004E204552524F52202020000024242424D6
:1012300047505320435243204552524F52202020C2
:1012400000002424242447505320434F4D4D554E35
:1012500049434154494F4E204552524F5200544544
:10126000535420444520000042414C4C4F4F4E20E7
:101270005041594C4F4144205620000020425920F3
:101280004F4D33424300547970652048454C5020FF
:10129000666F7220496E666F00004543484F00003C
:1012A0004D5943004D5943414C4C000054520000ED
:1012B00054524143450054584400545844454C410D
:1012C0005900554E5000554E50524F544F0044490E
:1012D00053500000444953504C41590048454C502C
:1012E0000000534552475053000054544558540091
:1012F0005441494C000053594D424F4C0000484F57
:101300004C4400005458540054585441494C000077
:101310005645520056455253494F4E004357494493
:101320000000435742415400435754454D5000007C
:1013300050524553530050524553535552450000A7
:10134000465251004652455155454E43590052466A
:101350005251000044455600444556494154494FB6
:101360004E0042415544000053504545440044421C
:1013700049545300534249545300424154560000CB
:1013800054454D500000504F55540000504F5745A4
:101390005200494453500000435753500000534FEC
:1013A0004C415200534F4C415243454C4C00524526
:1013B0004600444154410000534C454550005445BB
:1013C0005354000043414C49425241544500534557
:1013D000545000004E4F4750530055424C4F580058
:1013E0005254545900004F46465345540000455846
:1013F00049540000436F6D6D616E64206973206E07
:101400006F742076616C6964000043414C4942521C
:10141000415445204F4E00005345542046524551FB
:1014200055454E4359204F4E20504F5254412E3275
:1014300020544F203132303020487A007479706562
:1014400020552870292C2044286F776E292C205392
:10145000286176652920726573702E2045286E6498
:1014600029004D5943616C6C2000554E50726F74C9
:101470006F2000004652455155454E43593A2000D1
:101480004357202620525454592046524551554521
:101490004E43593A20005443584F20465245515527
:1014A000454E43593A200000504F574552204F5562
:1014B000543A2000444556494154494F4E3A200081
:1014C00053504545443A2000444154412042495438
:1014D000533A200053544F5020424954533A20006D
:1014E0004D4F44454D204F46465345543A20000049
:1014F000424154566F6C74616765200054454D50ED
:1015000065726174757265200000435753503A202C
:1015100000004357424154200000435754454D506A
:101520002000545844656C6179200000545854617F
:10153000696C200053594D424F4C2000484F4C4499
:10154000206F666620005452616365200000534F8F
:101550004C415220000055424C4F58200000505240
:101560004553535552452000534C454550200000EB
:1015700053455247505320003438303020426400E5
:101580003936303020426400313932303020426404
:101590000000457665727920000054544558542067
:1015A00000004D617820646576696174696F6E2012
:1015B0006973203130303020487A00004D61782046
:1015C00062617564726174652069732031303030F6
:1015D000204264004D617820646174612062697406
:1015E00073206973203800004D61782073746F7028
:1015F000206269747320697320320000564552538B
:10160000494F4E3A204243504C20762E000056421D
:1016100061743A20000054656D703A200000552036
:101620002D205057522055702C2044202D205057EB
:101630005220446F776E2C2045202D204578697408
:101640000000436F6D6D616E647320287769746864
:10165000206578616D706C65293A200044495350CB
:101660002020202020202D20446973706C61792077
:10167000616C6C20736574696E6773004D594361CA
:101680006C6C202020202D20286D7963616C6C20EB
:101690004F4D3342432D313129005452616365204F
:1016A000202020202D2028786D69742F6F666629F0
:1016B00020666F7220646562756767696E67206F68
:1016C0006E6C7900545844656C61792020202D207F
:1016D000747864656C6179206E20303C6E3C3130EA
:1016E0003020286E2078203130206D732900545826
:1016F0005461696C202020202D2054582074616989
:101700006C2074696D6520286E2078203130206D42
:1017100073290000554E50726F746F2020202D20C9
:1017200028756E70726F746F2061707273207620EE
:1017300077696465312D3129202D20332064696754
:101740006973206D6178000053594D424F4C202041
:1017500020202D203220415052532073796D626F2A
:101760006C73202D2064656661756C74206973202C
:1017700042414C4C4F4F4E20282F4F2900004652DB
:1017800051202020202020202D2066726571756553
:101790006E637920696E20487A00524652512020AB
:1017A000202020202D206672657175656E6379207A
:1017B000666F72205254545920696E20487A000096
:1017C000525454592020202020202D204F4E206F8D
:1017D00072204F4646004F46465345542020202055
:1017E0002D206D6F64656D206672657175656E6321
:1017F00079206F666673657420696E20487A2028A8
:101800006D61782E202B2D33303030302900444547
:1018100056202020202020202D20646576696174C8
:10182000696F6E20696E20487A004241554420203D
:10183000202020202D20626175647261746520660D
:101840006F722052545459207472616E736D6974B2
:1018500074696E67000044424954532020202020C0
:101860002D206E756D626572206F662064617461F3
:101870006269747300005342495453202020202091
:101880002D206E756D626572206F662073746F70A7
:101890006269747320312E35203D2031350042417C
:1018A00054562020202020202D2073656E64206255
:1018B000617465727920766F6C74616765202D2084
:1018C000594553206F72204E4F0054454D502020F3
:1018D000202020202D2073656E6420696E626F7851
:1018E0002074656D7065726174757265202D205964
:1018F0004553206F72204E4F0000504F57455220E5
:101900006F7220504F5554202D206F757470757470
:1019100020706F77657220696E206D570000524508
:1019200046202020202020202D20584F206F72207C
:101930005443584F206672657175656E63792069EE
:101940006E20487A20286D696E2E2031303030307C
:101950003030302C206D61782E20333230303030F2
:101960003030000055424C4F5820202020202D20A0
:101970004F4E203D2055424C4F582C204F4646207C
:101980003D205155454354454C00505245535375E5
:10199000726520202D204F4E203D20424D50313881
:1019A000302070726573656E742C204F4646203D62
:1019B000206E6F742070726573656E740000484FFE
:1019C0004C446F66662020202D20686F6C64206F69
:1019D00066662074696D6520696E206D696E757428
:1019E00065730000435749442020202020202D20EB
:1019F00073656E64204357206964656E7469666917
:101A00006572204F4E206F72204F464600004357AC
:101A100042415420202020202D2073656E642062D6
:101A2000617465727920766F6C7461676520696E88
:101A3000204357202D20594553206F72204E4F00D0
:101A4000435754454D50202020202D2073656E644F
:101A50002074656D706572617475726520696E20A1
:101A60004357202D20594553206F72204E4F0000C0
:101A700043575350206F722049445350202D2073F8
:101A800070656564206F66204357206964656E74D5
:101A9000696669657220696E2057504D0000534F8A
:101AA0004C415263656C6C202D206D6F756E7465B2
:101AB00064202D204F4E206F72206E6F74206D6F4A
:101AC000756E746564202D204F4646004543484F8F
:101AD0002020202020202D204F4E206F72204F46A6
:101AE0004600534C45455020202020202D20737760
:101AF0006974636820746865204750532072656379
:101B00006569766572202D204F4E206F72204F46FA
:101B10004600534552475053202020202D2062611B
:101B2000756472617465206F66204750532072653A
:101B3000636569766572202834383030206F7220F2
:101B400039363030206F7220313932303029000080
:101B500043414C494252415445202D2063616C69F8
:101B600062726174652031323030487A000044413D
:101B700054412020202020202D206964656E746946
:101B80006669636174696F6E206F66207261646953
:101B90006F20636869700000564552202020202085
:101BA00020202D20736F66747761726520766572D0
:101BB00073696F6E00004558495420202020202072
:101BC0002D20656E64206F6620636F6D6D616E649D
:101BD00020696E746572707265746572000054419C
:101BE000494C20287461696C20746578742065768E
:101BF000657279206E292D286F6E2C6F66662C6EAB
:101C0000292D6E3D30206973206F666620616E64F9
:101C100020313C6E3C39206576657279206E2D74DA
:101C200068206D657373616765005454455854208E
:101C3000202020202D207461696C20746578742028
:101C40002D20323530206368617273206D61780019
:101C50005461696C207465787420636F6D6D616E7A
:101C600064733A005C5520202020202020202D2065
:101C700073656E642062617465727920766F6C742E
:101C8000616765005C5620202020202020202D2028
:101C900073656E642073797374656D20766F6C74F0
:101CA000616765005C5320202020202020202D200B
:101CB00073656E6420736F6C617220766F6C7461F3
:101CC000676500005C4920202020202020202D2056
:101CD00073656E6420736F6C6172206375727265D8
:101CE0006E7400005C5420202020202020202D2015
:101CF00073656E6420696E7465726E616C207465C4
:101D00006D7065726174757265005C5820202020CA
:101D1000202020202D2073656E6420657874657204
:101D20006E616C2074656D706572617475726500AA
:101D30005C5720202020202020202D2073656E64F9
:101D400020726164696F636869702074656D706585
:101D500072617475726500005C5020202020202084
:101D600020202D2073656E64207072657373757208
:101D700065005C4620202020202020202D20736537
:101D80006E642074656D706572617475726520662D
:101D9000726F6D2070726573737572652073656EF6
:101DA000736F72005C4220202020202020202D20F4
:101DB00073656E64206E756D626572206F66207249
:101DC0006563656976656420736174656C6C6974BC
:101DD000657300005C5A20202020202020202D2028
:101DE000736F6674776172652076657273696F6E62
:101DF000000043686970205265766973696F6E3AB6
:101E00002000506172743A2053690000506172746E
:101E1000204275696C643A20307800004465736331
:101E200072697074696F6E2049643A2030780000DE
:101E3000437573746F6D65722049643A2030780081
:101E4000524F4D2049643A20307800005361766546
:101E5000643A20004E6F74207361766564202D20F3
:101E600041637475616C2076616C75653A20000081
:101E70004243545241434B200000415052532020D2
:101E8000000008000000090000000A0000000B002C
:101E900000000C0000000D0000000E00000010000B
:101EA00000001200000014000000170000001A00DB
:101EB00000001E00000022000000270000002D008E
:101EC000000036000000460000005E0000007F00B9
:101ED00000007F0000007F000000080000000900F3
:101EE00000000A0000000B0000000C0000000D00C4
:101EF00000000E000000100000001200000014009E
:101F00000000170000001A0000001E000000220060
:101F10000000270000002D000000360000004600F1
:101F200000005E0000007F0000007F0000007F00D6
:101F3000000008000000090000000A0000000B007B
:101F400000000C0000000D0000000E00000010005A
:101F500000001200000014000000170000001A002A
:101F600000001E00000022000000270000002D00DD
:101F7000000036000000460000005E0000007F0008
:101F800000007F0000007F000000400E3E6E006AEF
:101F9000A00EAF6E200EAC6E900EAB6EA00E756EE6
:101FA000200E726E900E716E0001AB0E926E9A0E44
:101FB000936E0F0E946EF40ED36ED26AC00E9B6EAB
:101FC000796A786AF26AF16AF06A816A010EC26E11
:101FD000080EC16EAB0EC06E0B0E0F01386F396B61
:101FE000080E3A6FE00E426F416F100E406F9E0E6A
:101FF0009C6E9D6AA06A040E9F6EA26A070ED56E43
:10200000460ECD6ECC6ABD6A2F0EBA6E140E516F9D
:102010004E6B4A6BC66A6C6AAC98AC84B886060E86
:10202000B06E800EAF6EAB9E708672987284060E94
:10203000766E800E756E718E01015B6B5C6B5D6BF5
:10204000596B5A6B00EE80F0EF6A00EE86F0EF6A93
:1020500000EE91F0EF6A00EE9CF0EF6A00EEA7F060
:10206000EF6A00EEB2F0EF6A00EEBDF0EF6A00EE4C
:10207000C8F0EF6A0401186B176B166B156B1A6BBF
:10208000196B036B106B0F6B94988B98949A8B8AD7
:102090005A0E010199630AD05A0E9A6307D05A0E5C
:1020A0009B6304D09C515A0A000102E0000E01D04B
:1020B000010E3B6E000E010156B7010E3B160001EA
:1020C0002BE0030E166EE80E63EC03F073EC44F0A5
:1020D0009A0E356E990E346E190E336E7F0E326E77
:1020E00014C439F013C438F012C437F011C436F0F8
:1020F000BAEC05F00108E5E001015E6B970E010105
:102100005E5D000109E2070E166ED00E63EC03F06F
:1021100001015E2B0001F2E35A0E01019C6F9B6FDF
:102120009A6F996F000193EC3BF0640E62EC03F040
:10213000949A8B8A020E166E580E63EC03F0949AF2
:102140008B9AE3C3FCF3E2C3FBF3E1C3FAF3E0C30E
:10215000F9F362EC3EF0C80E62EC03F0070E0301E7
:10216000876F020E886F010E896F8A6FFCC38BF335
:10217000FBC38CF3FAC38DF3F9C38EF3000147EC74
:1021800043F0140E62EC03F0040E0301876F200E7F
:10219000886F896B8A6B8B6B000147EC43F0140EE0
:1021A00062EC03F0080E0301876F130E886F040EB4
:1021B000896F150E8A6F210E8B6F200E8C6F080EA3
:1021C0008D6F0B0E8E6F8F6B000147EC43F04EEC62
:1021D0004CF02EEC21F0080E0301DB250101606FAD
:1021E000050E0301876F110E886F200E896F010E97
:1021F0008A6F510E8B6F60C18CF3000145EC43F088
:10220000060E0301876F110E886F200E896F020E74
:102210008A6F0D0E8B6F8C6B8D6B000145EC43F05C
:10222000050E0301876F110E886F220E896F010E54
:102230008A6F8B6B080E8C6F000145EC43F050ECFD
:1022400020F00401026B00015FEC20F0050E030199
:10225000876F110E886F896B010E8A6F8B6F8C6F81
:10226000000145EC43F00C0E0301876F110E886FDF
:10227000200E896F080E8A6F180E8B6F010E8C6FFF
:102280008D6B080E8E6F020E8F6F800E906F916BAC
:10229000F00E926F100E936F000145EC43F00D0E9F
:1022A0000301876F110E886F200E896F090E8A6FE8
:1022B000220E8B6F8C6B820E8D6F030E8E6FEE0E67
:1022C0008F6FA20E906F020E916F5D0E926F020ED5
:1022D000936F946B000145EC43F00C0E0301876F84
:1022E000110E886F200E896F080E8A6F420E8B6F59
:1022F000A40E8C6F030E8D6FD60E8E6F030E8F6F34
:10230000906BF50E916F010E926F800E936F00012E
:1023100045EC43F0100E0301876F110E886F210EFC
:10232000896F0C0E8A6F8B6BA20E8C6F810E8D6F76
:10233000260E8E6FAF0E8F6F3F0E906FEE0E916F69
:10234000C80E926FC70E936FDB0E946FF20E956FEF
:10235000020E966F080E976F000145EC43F0100EC9
:102360000301876F110E886F210E896F0C0E8A6F23
:102370008B6F070E8C6F030E8D6F150E8E6FFC0E1C
:102380008F6F0F0E906F916BA20E926F810E936FF5
:10239000260E946FAF0E956F3F0E966FEE0E976FF1
:1023A000000145EC43F0100E0301876F110E886F9A
:1023B000210E896F0C0E8A6F180E8B6FC80E8C6FF2
:1023C000C70E8D6FDB0E8E6FF20E8F6F020E906F49
:1023D000080E916F070E926F030E936F150E946F98
:1023E000FC0E956F0F0E966F976B000145EC43F056
:1023F000080E0301876F110E886F220E896F040E7D
:102400008A6F8B6B080E8C6F7F0E8D6F8E6B3D0EFF
:102410008F6F000145EC43F00B0E0301876F110E27
:10242000886F230E896F070E8A6F8B6B2C0E8C6F53
:102430000E0E8D6F0B0E8E6F040E8F6F0C0E906F45
:10244000730E916F030E926F000145EC43F032EC76
:1024500020F08BEC20F0320E62EC03F077EC20F0F1
:1024600044EF24F0010156510001E8AA02D050ECDB
:102470004EF016EC47F0719E010156510001E8A89C
:102480002BD2800E026E400E096E226A3DC421F0EE
:10249000066A056A200E016EB50EA5EC01F0620E0B
:1024A000A5EC01F0060EA5EC01F03B0EA5EC01F049
:1024B0002C0EA5EC01F0000EA5EC01F0010EA5EC30
:1024C00001F0060EA5EC01F0000EA5EC01F0000EE7
:1024D000A5EC01F0200EA5EC01F0900EA5EC01F0AA
:1024E000000EA5EC01F0000EA5EC01F0000EA5EC2D
:1024F00001F0000EA5EC01F0000EA5EC01F0000EBD
:10250000A5EC01F0000EA5EC01F0800E026E400E6D
:10251000096E226A3DC421F0066A056A200E016E2A
:10252000000EA5EC01F0000EA5EC01F0000EA5ECEC
:1025300001F0000EA5EC01F0000EA5EC01F0000E7C
:10254000A5EC01F0000EA5EC01F0000EA5EC01F0E9
:10255000000EA5EC01F0000EA5EC01F0000EA5ECBC
:1025600001F02C0EA5EC01F0010EA5EC01F0000E1F
:10257000A5EC01F0000EA5EC01F04F0EA5EC01F06A
:10258000C10EA5EC01F0030EA5EC01F0000EA5ECC8
:1025900001F0800E026E400E096E226A3DC421F0E9
:1025A000066A056A200E016E860EA5EC01F0020E89
:1025B000A5EC01F0000EA5EC01F0000EA5EC01F079
:1025C000FE0EA5EC01F0000EA5EC01F0000EA5EC4E
:1025D00001F0000EA5EC01F0640EA5EC01F0400E38
:1025E000A5EC01F0010EA5EC01F0000EA5EC01F048
:1025F0008F0EA5EC01F0870EA5EC01F0640E62ECE5
:1026000003F0800E026E400E096E226A3DC421F076
:10261000066A056A200E016EB50EA5EC01F0620E89
:10262000A5EC01F0060EA5EC01F0160EA5EC01F0EC
:10263000080EA5EC01F0000EA5EC01F0000EA5ECD3
:1026400001F0030EA5EC01F0030EA5EC01F0000E65
:10265000A5EC01F0510EA5EC01F0A20EA5EC01F0E5
:10266000060EA5EC01F0000EA5EC01F0230EA5EC82
:1026700001F0E70EA5EC01F0640E62EC03F0800EB1
:10268000026E400E096E226A3DC421F0066A056A98
:10269000200E016EB50EA5EC01F0620EA5EC01F066
:1026A000060EA5EC01F0110EA5EC01F0020EA5EC52
:1026B00001F0000EA5EC01F0080EA5EC01F0010EF2
:1026C000A5EC01F0220EA5EC01F0920EA5EC01F0B4
:1026D000B50EA5EC01F0620EA5EC01F0060EA5EC1E
:1026E00001F0090EA5EC01F00D0EA5EC01F0000EB5
:1026F000A5EC01F0000EA5EC01F0000EA5EC01F038
:10270000000EA5EC01F0000EA5EC01F0FF0EA5EC0B
:1027100001F0FF0EA5EC01F0000EA5EC01F0000E9B
:10272000A5EC01F0000EA5EC01F0000EA5EC01F007
:10273000000EA5EC01F0000EA5EC01F0070EA5ECD3
:1027400001F0210EA5EC01F0AF0EA5EC01F0640E36
:1027500062EC03F0800E026E400E096E226A3DC4E8
:1027600021F0066A056A200E016E100EF76EA40EA7
:10277000F66E0900F55003E0A5EC01F0FAD70D0E56
:10278000A5EC01F00A0EA5EC01F0640E62EC03F07A
:10279000800E026E400E096E226A3DC421F0066A68
:1027A000056A200E016E100EF76EBC0EF66E090063
:1027B000F55003E0A5EC01F0FAD70D0EA5EC01F001
:1027C0000A0EA5EC01F0640E62EC03F0800E026EBE
:1027D000400E096E226A3DC421F0066A056A200E89
:1027E000016E100EF76ED40EF66E0900F55003E080
:1027F000A5EC01F0FAD70D0EA5EC01F00A0EA5EC40
:1028000001F0640E62EC03F0800E026E400E096E61
:10281000226A3DC421F0066A056A200E016E100E80
:10282000F76EEC0EF66E0900F55003E0A5EC01F032
:10283000FAD70D0EA5EC01F00A0EA5EC01F0640E1E
:1028400062EC03F0800E026E400E096E226A3DC4F7
:1028500021F0066A056A200E016E110EF76E040E55
:10286000F66E0900F55003E0A5EC01F0FAD70D0E65
:10287000A5EC01F00A0EA5EC01F0640E62EC03F089
:10288000800E026E400E096E226A3DC421F0066A77
:10289000056A200E016E110EF76E1C0EF66E090011
:1028A000F55003E0A5EC01F0FAD70D0EA5EC01F010
:1028B0000A0EA5EC01F0DDEC53F001015A510001C4
:1028C000E8A602D0DDEC53F001015A510001E8A660
:1028D00002D0DDEC53F01BD0800E026E400E096E6C
:1028E000226A3DC421F0066A056A200E016E110EAF
:1028F000F76E340EF66E0900F55003E0A5EC01F01A
:10290000FAD70D0EA5EC01F00A0EA5EC01F00401BA
:10291000346B140E336F640E356F3B6B000116D1B0
:10292000030E04013B5D000106E2EA0E166E600E26
:1029300063EC03F00BD1010156510001E8A45CD017
:10294000010156510001E8B81CD0800E026E400E05
:10295000096E226A3DC421F0066A056A200E016EE6
:10296000110EF76E660EF66E0900F55003E0A5EC49
:1029700001F0FAD70D0EA5EC01F00A0EA5EC01F05E
:102980003BD0800E026E400E096E226A3DC421F0DB
:10299000066A056A200E016EB50EA5EC01F0620E06
:1029A000A5EC01F0060EA5EC01F0570EA5EC01F028
:1029B000080EA5EC01F0000EA5EC01F0010EA5EC4F
:1029C00001F0000EA5EC01F0000EA5EC01F0000EE8
:1029D000A5EC01F0500EA5EC01F04F0EA5EC01F0B6
:1029E000540EA5EC01F0530EA5EC01F0AC0EA5ECD5
:1029F00001F0850EA5EC01F0A20ED36ED2889B9C4F
:102A0000C29001019553000109E001019507010EF3
:102A1000166ED50E63EC03F00001F3D7010E166EAF
:102A2000490E63EC03F09B8CD298F40ED36EC280F7
:102A30002C0ED2EC02F00101956F95075651000162
:102A4000E8A617D0B2EC44F018C435F017C434F03F
:102A500016C433F015C432F0396A386A376A7E0E0C
:102A6000366EBAEC05F0010804E0D8900101953704
:102A7000952B010156510001E8A45CD0010156518B
:102A80000001E8B81CD0800E026E400E096E226A6A
:102A90003DC421F0066A056A200E016E110EF76E24
:102AA000740EF66E0900F55003E0A5EC01F0FAD7BC
:102AB0000D0EA5EC01F00A0EA5EC01F03BD0800E46
:102AC000026E400E096E226A3DC421F0066A056A54
:102AD000200E016EB50EA5EC01F0620EA5EC01F022
:102AE000060EA5EC01F0570EA5EC01F0080EA5ECC2
:102AF00001F0000EA5EC01F0010EA5EC01F0000EB6
:102B0000A5EC01F0000EA5EC01F0000EA5EC01F023
:102B1000200EA5EC01F04E0EA5EC01F0550EA5EC33
:102B200001F0520EA5EC01F07B0EA5EC01F0C30EF6
:102B3000A5EC01F0130E166E880E63EC03F0010194
:102B40009453000102E001019407000122D8030E12
:102B500004013B5D000106E34E0E166E200E63EC91
:102B600003F017D801019453000105E12A0ED2ECBD
:102B700002F00101946F000E010156B1010E3B6E8F
:102B8000000E56BF010E3B120001D8A4C9EC54F050
:102B9000C7D6010156510001E8AC0AD001EE9DF004
:102BA000110EF76E800EF66E89EC04F0EE6A02D11B
:102BB00004014D6B010156510001E8B837D0800E79
:102BC000026E800E096E226A3DC421F00B0E066E65
:102BD000B80E056E63EC01F0D8A08DEF1CF0240850
:102BE000F9E163EC01F0D8A08DEF1CF04708F2E1A9
:102BF00063EC01F0D8A08DEF1CF05008EBE163EC22
:102C000001F0D8A08DEF1CF04708E4E163EC01F07F
:102C1000D8A08DEF1CF04708DDE163EC01F0D8A0EF
:102C20008DEF1CF00101606F000135D0800E026E47
:102C3000800E096E226A3DC421F00B0E066EB80E9E
:102C4000056E63EC01F0D8A08DEF1CF02408F9E1CB
:102C500063EC01F0D8A08DEF1CF04708F2E163ECC3
:102C600001F0D8A08DEF1CF04E08EBE163EC01F011
:102C7000D8A08DEF1CF04708E4E163EC01F0D8A088
:102C80008DEF1CF04708DDE163EC01F0D8A08DEF7B
:102C90001CF00101606F0001010E486E60C149F235
:102CA000800E026E800E096E226A3DC421F0066A13
:102CB000C80E056E63EC01F0D8A07CD70101606FEF
:102CC00002EE49F04850E926000EEA2260C1EFFF0B
:102CD000482A2A0E605DD8A4010E3B6E4F0E485C58
:102CE000010ED8B0000E3B160001DAE1800E026E34
:102CF000800E096E226A3DC421F0050E3A6E020E66
:102D0000086E08EC00F00101776F02EE49F04850C0
:102D1000E926000EEA22EF6A56510001E8B814D005
:102D200001EE9DF0470EEE6E500EEE6E470EEE6E0B
:102D3000EE6E12EE49F0000EE75204E0E6CFEEFF31
:102D4000E82EFAD7EF6A13D001EE9DF0470EEE6E33
:102D50004E0EEE6E470EEE6EEE6E12EE49F0000E67
:102D6000E75204E0E6CFEEFFE82EFAD7EF6A010162
:102D70005E6B04012F6B000101EE9DF001015E51BD
:102D8000EB500C6E2A0E0C5C00010CE001EE9DF085
:102D900001015E51EB500C6E04012F1B01015E2BF3
:102DA0000001E9D704012F510101775D0001D8A48A
:102DB000B3EF1CF0010156510001E8AC0AD001EE5E
:102DC000F3F0110EF76ECE0EF66E89EC04F0EE6A9B
:102DD00002D1010156510001E8B837D0800E026ED1
:102DE000800E096E226A3DC421F00B0E066EB80EED
:102DF000056E63EC01F0D8A08DEF1CF02408F9E11A
:102E000063EC01F0D8A08DEF1CF04708F2E163EC11
:102E100001F0D8A08DEF1CF05008EBE163EC01F05D
:102E2000D8A08DEF1CF05608E4E163EC01F0D8A0C7
:102E30008DEF1CF05408DDE163EC01F0D8A08DEFBC
:102E40001CF00101606F000135D0800E026E800E13
:102E5000096E226A3DC421F00B0E066EB80E056E97
:102E600063EC01F0D8A08DEF1CF02408F9E163ECCD
:102E700001F0D8A08DEF1CF04708F2E163EC01F0FF
:102E8000D8A08DEF1CF04E08EBE163EC01F0D8A068
:102E90008DEF1CF05608E4E163EC01F0D8A08DEF53
:102EA0001CF05408DDE163EC01F0D8A08DEF1CF0BC
:102EB0000101606F0001010E486E60C149F2800E91
:102EC000026E800E096E226A3DC421F0066AC80EA9
:102ED000056E63EC01F0D8A06DD70101606F02EEC2
:102EE00049F04850E926000EEA2260C1EFFF482A67
:102EF0002A0E605DD8A4010E3B6E4F0E485C010E99
:102F0000D8B0000E3B160001DAE1800E026E800E92
:102F1000096E226A3DC421F0050E3A6E020E086E5B
:102F200008EC00F00101776F02EE49F04850E92605
:102F3000000EEA22EF6A56510001E8B815D001EE02
:102F4000F3F0470EEE6E500EEE6E560EEE6E540E11
:102F5000EE6E12EE49F0000EE75204E0E6CFEEFF0F
:102F6000E82EFAD7EF6A14D001EEF3F0470EEE6EBA
:102F70004E0EEE6E560EEE6E540EEE6E12EE49F0E2
:102F8000000EE75204E0E6CFEEFFE82EFAD7EF6A34
:102F900001015E6B04012F6B000101EEF3F00101F2
:102FA0005E51EB500C6E2A0E0C5C00010CE001EE41
:102FB000F3F001015E51EB500C6E04012F1B010177
:102FC0005E2B0001E9D704012F510101775D00015B
:102FD000D8A4EAEF1CF002EE49F011EEF3F0550E22
:102FE000E75204E0E6CFEEFFE82EFAD7EF6A0301DE
:102FF0004B6B4A6B4D6B4C6B01015F6B000159ECE5
:1030000021F003EE54F0EECFF3FFEFCFF4FFF450D6
:10301000F31006E101017C6B7B6B7A6B000121D020
:1030200003EE54F004EC00F003014A6F1AC04BF3B6
:103030004BC312F04AC311F0000E9FEC03F00101E4
:103040007C6F4BC312F04AC311F0010E9FEC03F0EA
:103050007B6F4BC312F04AC311F0020E9FEC03F0DA
:103060007A6F01015F6B00015FEC21F003EE54F019
:10307000EECFF3FFEFCFF4FFF450F31007E1300E83
:1030800001017F6F7E6F7D6F000121D003EE54F050
:1030900004EC00F003014C6F1AC04DF34DC312F065
:1030A0004CC311F0000E9FEC03F001017F6F4DC384
:1030B00012F04CC311F0010E9FEC03F07E6F4DC374
:1030C00012F04CC311F0020E9FEC03F07D6F04016F
:1030D000396B02EE49F011EE9DF0550EE75204E017
:1030E000E6CFEEFFE82EFAD7EF6A01015F6B000131
:1030F0005AEC21F003015451C96F300EC95D000133
:10310000D8B46AEF1CF001015F6B00015EEC21F0A6
:10311000030154510101846F030155510101856F71
:10312000030156510101866F030157510101876F59
:10313000030158510C6E2E0E0C5C000102E00101DF
:103140005A87030159510101886F03015A51010146
:10315000896F0F0E8415606F605111EC08F0396AA9
:10316000386A200E376E820E366E6AEC07F035C074
:10317000C4F334C0C3F333C0C2F332C0C1F30F0E83
:103180008515606F605111EC08F0C4C339F0C3C3FA
:1031900038F0C2C337F0C1C336F076EC06F035C064
:1031A000C4F334C0C3F333C0C2F332C0C1F30F0E53
:1031B0008615606F6051640DF3CF67F1F4CF68F14D
:1031C0000F0E8715606F60510A0DF3CF60F16051EB
:1031D0006727000E68230F0E8815606F6051672700
:1031E000000E6823396A386A160E376E880E366EFE
:1031F00068C133F067C132F013EC08F004EC07F05B
:1032000035C027F034C026F033C025F032C024F09A
:10321000C4C339F0C3C338F0C2C337F0C1C336F0FA
:1032200027C035F026C034F025C033F024C032F07A
:1032300076EC06F035C0C4F334C0C3F333C0C2F338
:1032400032C0C1F35F6B00015DEC21F0030154510A
:103250000C6E4E0E0C5C000104E101015C83000168
:1032600025D0030154510C6E530E0C5C00011CE17F
:1032700001015C93356A346A800E336E7F0E326EC4
:10328000C4C339F0C3C338F0C2C337F0C1C336F08A
:103290006AEC07F035C0C4F334C0C3F333C0C2F3E3
:1032A00032C0C1F3000102D001015A8701015F6BF6
:1032B00000015CEC21F0030154510C6E0F0E0C1454
:1032C00001018A6F256A8AC124F025500A0DF3CFC7
:1032D00025F024500A0DF3CF24F0F45025260301E5
:1032E00055510C6E296A0CC028F00F0E2816000EDE
:1032F00029162450282401018A6F256A8AC124F0E6
:1033000025500A0DF3CF25F024500A0DF3CF24F0F9
:10331000F4502526030156510C6E296A0CC028F082
:103320000F0E2816000E29162450282401018A6F3A
:10333000030157510C6E0F0E0C1401018B6F256A9F
:103340008BC124F025500A0DF3CF25F024500A0D2F
:10335000F3CF24F0F4502526030158510C6E296A4E
:103360000CC028F00F0E2816000E29162450282411
:1033700001018B6F03015A510C6E0F0E0C140101E9
:103380008C6F8A5111EC08F035C027F034C026F05C
:1033900033C025F032C024F08B5111EC08F035C059
:1033A0002BF034C02AF033C029F032C028F0356A3F
:1033B000346A200E336E820E326E2BC039F02AC072
:1033C00038F029C037F028C036F06AEC07F035C075
:1033D0002BF034C02AF033C029F032C028F08C51D1
:1033E00011EC08F02BC039F02AC038F029C037F0B2
:1033F00028C036F076EC06F035C02BF034C02AF049
:1034000033C029F032C028F0396A386A160E376E98
:10341000880E366E2BC035F02AC034F029C033F048
:1034200028C032F004EC07F035C02BF034C02AF08D
:1034300033C029F032C028F027C039F026C038F058
:1034400025C037F024C036F02BC035F02AC034F048
:1034500029C033F028C032F076EC06F035C0C8F34E
:1034600034C0C7F333C0C6F332C0C5F3256A8CC17C
:1034700024F025500A0DF3CF25F024500A0DF3CF88
:1034800024F0F450252603015B510C6E296A0CC010
:1034900028F00F0E2816000E2916245028240101AA
:1034A0008C6F5F6B00015BEC21F0030154510C6EDB
:1034B000450E0C5C000104E101015C95000125D082
:1034C000030154510C6E570E0C5C00011CE101010C
:1034D0005C85356A346A800E336E7F0E326EC8C3E7
:1034E00039F0C7C338F0C6C337F0C5C336F06AEC4D
:1034F00007F035C0C8F334C0C7F333C0C6F332C0D9
:10350000C5F3000102D001015A8701015F6B000180
:1035100059EC21F003EE4EF013EE54F0320EE75268
:1035200004E0E6CFEEFFE82EFAD7EF6A03EE4EF0A6
:1035300004EC00F004013B6F01015F6B000157ECEC
:1035400021F001EE3DF013EE54F0320EE75204E0AC
:10355000E6CFEEFFE82EFAD7EF6A01EE3DF004EC7D
:1035600000F00401336F1AC034F4256A7BC124F0E3
:103570000F0E2416000E2516296A0A0E286E2D6AD3
:103580007AC12CF00F0E2C16000E2D1629C01AF041
:103590002850196E2C02F3CF28F0F4CF29F01A50DE
:1035A0002C02F350292619502D02F35029262450BD
:1035B000282401017B6F0A0E7B5D000105E21C0ED1
:1035C00001017B27000103D06C0E01017B27000164
:1035D000256A7DC124F00F0E2416000E2516296AD7
:1035E0000A0E286E2D6A7CC12CF00F0E2C16000ED0
:1035F0002D1629C01AF02850196E2C02F3CF28F08E
:10360000F4CF29F01A502C02F350292619502D021C
:10361000F35029262450282401017D6F200E7D2798
:10362000256A7EC124F00F0E2416000E2516296A85
:103630000A0E286E2D6A7FC12CF00F0E2C16000E7C
:103640002D1629C01AF02850196E2C02F3CF28F03D
:10365000F4CF29F01A502C02F350292619502D02CC
:10366000F3502926245028247F6F1C0E7F27200E1C
:103670008427200E85275C510001E8A203D0200E8C
:1036800001018727650E01018A5D000103E3200E19
:103690000101882701015C510001E8A403D0200E3C
:1036A00001018927650E01018A5D000105E36C0EA9
:1036B00001018A2700010DD00A0E01018A5D000177
:1036C00005E31C0E01018A27000103D0760E0101DB
:1036D0008A270A0E01018B5D000105E2580E0101E7
:1036E0008B27000103D01C0E01018B270001BBC3F7
:1036F0000CF0BCC30DF00DC0BAF30CC0B9F3BDC3E0
:103700000CF0BEC30DF00DC0BCF30CC0BBF3BFC3C7
:103710000CF0C0C30DF00DC0BEF30CC0BDF334C43B
:10372000C0F333C4BFF3BFC30CF0C0C30DF0BDC3BF
:103730000EF0BEC30FF00E500C5C0F500D5802E39C
:10374000000E01D0010E3B6EBDC30CF0BEC30DF0E8
:10375000BBC30EF0BCC30FF00E500C5C0F500D58E5
:1037600002E3000E01D0010E3B16BBC30CF0BCC33C
:103770000DF0B9C30EF0BAC30FF00E500C5C0F5031
:103780000D5802E3000E01D0010E3B160FE00101BF
:10379000859B050E0401345D000108E305E1DD0EA3
:1037A0000401335D000102E301015B83010E0401AA
:1037B000345D000108E305E12C0E0401335D0001D6
:1037C00002E3000E01D0010E3B6E000E01015BB35F
:1037D000010E3B16000105E001015D8100013AEF99
:1037E0001EF01C0E01018C2784C157F085C158F0D2
:1037F00086C159F087C15AF088C15BF089C15CF07D
:103800005D6A8AC149F28BC14AF28CC14BF27BC11D
:103810004CF27DC14DF27FC14EF28EC14FF28DC18F
:1038200050F2100E040133250101716F270E0401BF
:1038300034210101726F72C112F071C111F0200EBA
:10384000166E590E156ED7EC03F0246E12C025F0DB
:10385000210E24240C6E0CC051F272C112F071C101
:1038600011F0200E166E590E156ED7EC03F01AC02B
:1038700072F119C071F172C112F071C111F0166AC2
:103880005B0E156ED7EC03F0246E12C025F0210EEE
:1038900024240C6E0CC052F272C112F071C111F0EE
:1038A000166A5B0E156ED7EC03F01AC025F019C02E
:1038B00024F0210E24240C6E0CC053F27D0E020164
:1038C000546F0D0E556F0401396B000182EC47F007
:1038D0002AEF23F004014D2B070E4D5D000115E387
:1038E00000EEE9F00D0EEE6E0A0EEE6E110EF76EA2
:1038F000F40EF66E89EC04F00D0EEE6E0A0EEE6E0E
:10390000EE6A53EC57F004014D6B0001270E166E62
:10391000100E63EC03F0DAEF15F0949494948B940A
:10392000640E62EC03F094840401392B060E395DB9
:10393000000117E300EEE9F00D0EEE6E0A0EEE6EDA
:10394000120EF76E0C0EF66E89EC04F00D0EEE6E94
:103950000A0EEE6EEF6A0401396B000153EC57F06A
:1039600070D0C9EF15F00401392B060E395D000146
:103970002FE300EEE9F00D0EEE6E0A0EEE6E120E63
:10398000F76E2C0EF66E89EC04F011EE9DF0550EDC
:10399000E75204E0E6CFEEFFE82EFAD7020E016E02
:1039A000086E0101775189EC00F0200EEE6E020ED8
:1039B000016E086E04012F5189EC00F00D0EEE6EC1
:1039C0000A0EEE6EEF6A396B000153EC57F039D0F6
:1039D000C9EF15F00401392B060E395D00012FE304
:1039E00000EEE9F00D0EEE6E0A0EEE6E120EF76EA0
:1039F0002C0EF66E89EC04F011EEF3F0550EE75242
:103A000004E0E6CFEEFFE82EFAD7020E016E086E54
:103A10000101775189EC00F0200EEE6E020E016E6E
:103A2000086E04012F5189EC00F00D0EEE6E0A0EA7
:103A3000EE6EEF6A396B000153EC57F002D0DAEF0B
:103A400016F03DC457F44B0E04013D6F0101565171
:103A50000001E8B831D0800E026E800E096E226A35
:103A60003DC421F00B0E066EB80E056E63EC01F03E
:103A7000D8A053D72408FAE163EC01F0D8A04DD7C1
:103A80004708F4E163EC01F0D8A047D75008EEE115
:103A900063EC01F0D8A041D74708E8E163EC01F0FE
:103AA000D8A03BD74708E2E163EC01F0D8A035D7B6
:103AB0000101606F00012FD0800E026E800E096E32
:103AC000226A3DC421F00B0E066EB80E056E63EC43
:103AD00001F0D8A022D72408FAE163EC01F0D8A0C5
:103AE0001CD74708F4E163EC01F0D8A016D74E08C4
:103AF000EEE163EC01F0D8A010D74708E8E163ECF1
:103B000001F0D8A00AD74708E2E163EC01F0D8A0A1
:103B100004D70101606F0001010E486E60C149F2D7
:103B2000800E026E800E096E226A3DC421F0066A84
:103B3000C80E056E63EC01F0D8A088D70101606F54
:103B400002EE49F04850E926000EEA2260C1EFFF7C
:103B5000482A2A0E605DD8A4010E3B6E4F0E485CC9
:103B6000010ED8B0000E3B160001DAE1800E026EA5
:103B7000800E096E226A3DC421F0050E3A6E020ED7
:103B8000086E08EC00F00101776F02EE49F0485032
:103B9000E926000EEA22EF6A56510001E8B814D077
:103BA00001EE9DF0470EEE6E500EEE6E470EEE6E7D
:103BB000EE6E12EE49F0000EE75204E0E6CFEEFFA3
:103BC000E82EFAD7EF6A13D001EE9DF0470EEE6EA5
:103BD0004E0EEE6E470EEE6EEE6E12EE49F0000ED9
:103BE000E75204E0E6CFEEFFE82EFAD7EF6A0101D4
:103BF0005E6B04012F6B000101EE9DF001015E512F
:103C0000EB500C6E2A0E0C5C00010CE001EE9DF0F6
:103C100001015E51EB500C6E04012F1B01015E2B64
:103C20000001E9D704012F510101775D000106E190
:103C300004013D2B3D2B0001C9EF15F004013D2B84
:103C4000630E3D5D0001D8A001D700EEE9F00D0E36
:103C5000EE6E0A0EEE6E120EF76E420EF66E89ECE6
:103C600004F00D0EEE6E0A0EEE6EEE6A53EC57F097
:103C7000D5EF0FF0939A8A9A04DA6DEC20F00101E7
:103C80005E6B060E01015E5D00010EE200EE4EF07D
:103C900001015E51EB500C6E200E0C5C000104E043
:103CA00001015E2B0001EDE303EE54F0120EF76EFE
:103CB0005E0EF66E89EC04F010EE4EF001015E51DE
:103CC000E6CFEEFFE82EFCD72F0EEE6E410EEE6E25
:103CD0004D0EEE6EEE6A5E6B000103EE54F00101D4
:103CE0005E51EB500C6E0C5200010DE003EE54F0EF
:103CF00001015E51EB500401026F000138D901014E
:103D00005E2B0001E9D704013151050DF3CF15F009
:103D1000F4CF16F064EC03F002EE49F011EE9DF0E2
:103D2000550EE75204E0E6CFEEFFE82EFAD7EF6A31
:103D30000001D3EC3FF0030E166EE80E63EC03F0C7
:103D400001015E6B000103EE54F001015E51EB5086
:103D50000C6E0C5200010DE003EE54F001015E51B7
:103D6000EB500401026F000102D901015E2B00013A
:103D7000E9D701015D310001D8A083D0060E03010F
:103D8000876F110E886F200E896F020E8A6F0D0EDD
:103D90008B6F8C6B8D6B000145EC43F0030E166E40
:103DA000E80E63EC03F05ED9130E166E880E63EC1A
:103DB00003F000EEE9F0EF6A01015F6B00015EECD9
:103DC00021F000EEE9F013EE54F0320EE75204E079
:103DD000E6CFEEFFE82EFAD7EF6A01015F6B000134
:103DE0005DEC21F000EEE9F0EE50FEE1ED522C0E1C
:103DF000EE6E13EE54F0320EE75204E0E6CFEEFF23
:103E0000E82EFAD7EF6A01015F6B00015CEC21F04C
:103E100000EEE9F0EE50FEE1ED522C0EEE6E13EEE8
:103E200054F0320EE75204E0E6CFEEFFE82EFAD768
:103E3000EF6A01015F6B00015BEC21F002EE49F0DB
:103E400010EEE9F0230EE75204E0E6CFEEFFE82E95
:103E5000FAD72C0EEE6E13EE54F0320EE75204E059
:103E6000E6CFEEFFE82EFAD70D0EEE6EEF6A0101F7
:103E7000559D0001A9EC21F0240E4A6E31EF23F08C
:103E800075D001015731000132E373EC44F0030EA9
:103E9000166EE80E63EC03F003EE54F0200EEE6EA7
:103EA000550EEE6E10EE9CF00A0EE75204E0E6CFDF
:103EB000EEFFE82EFAD7560EEE6EEE6A01015E6B4B
:103EC000000103EE54F001015E51EB500C6E0C52F8
:103ED00000010DE003EE54F001015E51EB500401CE
:103EE000026F000144D801015E2B0001E9D70101F6
:103EF00057510001E8A239D0C3EC43F091510C6E48
:103F00002D0E0C5C02E14E0E916F030E166EE80E44
:103F100063EC03F003EE54F0200EEE6E540EEE6EE2
:103F200010EE91F00A0EE75204E0E6CFEEFFE82E25
:103F3000FAD7430EEE6EEE6A01015E6B000103EEEE
:103F400054F001015E51EB500C6E0C5200010DE07B
:103F500003EE54F001015E51EB500401026F0001C9
:103F600006D801015E2B0001E9D7C1D81200200E4E
:103F70000401025D00010BE104013151050DF3CF95
:103F800015F0F4CF16F064EC03F000011200410EBE
:103F90000401025D000112E2256A470E04010225B8
:103FA000246ED8B0252A2E0E245C046FAA6A04C49D
:103FB000A9FFD4EC02F0016F000110D0256A570E62
:103FC00004010225246ED8B0252A410E245C046F1A
:103FD000AA6A04C4A9FFD4EC02F0016F04010151E4
:103FE0000001E8BE25D0020E0401015D000120E3BE
:103FF000939A8A8A0401013100010BE304013151D3
:10400000030DF3CF15F0F4CF16F064EC03F00001CC
:1040100004D00401315162EC03F00001939A8A9AB2
:104020000401315162EC03F0D89001330001D6D77E
:1040300004013151020DF3CF15F0F4CF16F064EC0A
:1040400003F000011200050E0301876F110E886F47
:10405000200E896F010E8A6F8B6B8A0E8C6F0001A8
:1040600045EF43F0050E0301876F110E886F200E98
:10407000896F010E8A6F8B6B880E8C6F000145EF84
:1040800043F0050E0301876F110E886F200E896FB4
:10409000010E8A6F8B6B890E8C6F000145EF43F028
:1040A000050E0301876F110E886F220E896F010EB6
:1040B0008A6F8B6F01C48CF3000145EF43F0050E4E
:1040C0000301876F110E886F896B010E8A6F8B6BEE
:1040D00002C48CF3000145EF43F0020E0301876F29
:1040E000340E886F070E896F000145EF43F0020E12
:1040F0000301876F340E886F010E896F000145EF51
:1041000043F0020E0301876F340E886F050E896F2E
:10411000000145EF43F0060E0301876F310E886FF3
:10412000010E896F300E8A6F8B6B8C6B8D6B00016B
:1041300045EF43F0020E0301876F340E886F030EC4
:10414000896F000145EF43F0020E0301876F340EC3
:10415000886F080E896F000145EF43F0020E0301DE
:10416000876F340E886F060E896F000145EF43F0AC
:10417000020E0301876F340E886F020E896F0001F3
:1041800045EF43F0060E0301876F110E886F200E76
:10419000896F020E8A6F0D0E8B6FFEC38CF3FDC309
:1041A0008DF3000145EF43F0D5C327F0D4C326F0CB
:1041B000D3C325F0D2C324F02B6A800E2A6E5E0E84
:1041C000296E880E286E356A346A336A7F0E326E25
:1041D0002BC039F02AC038F029C037F028C036F09B
:1041E00076EC06F035C02BF034C02AF033C029F04D
:1041F00032C028F02852D8B43E84D8A4280627C05C
:1042000039F026C038F025C037F024C036F02BC076
:1042100035F02AC034F029C033F028C032F06AECFF
:1042200007F0B8EC07F00401096F33C00AF40AC4C0
:1042300000F409C4FFF3070E0301876F110E886FA6
:10424000200E896F030E8A6F0A0E8B6F8C6B00C471
:104250008DF3FFC38EF3000145EF43F0070E03011A
:10426000876F110E886F200E896F030E8A6F0A0EFA
:104270008B6F8C6B8D6B8E6B000145EF43F0080EDE
:104280000301876F130E886F040E896F150E8A6FF6
:10429000210E8B6F200E8C6F080E8D6F0B0E8E6FA4
:1042A0008F6B140E62EC03F0000147EF43F033D83C
:1042B00032D831D830D82FD82ED82DD82CD82BD8CA
:1042C00001015E6B000102EE49F001015F51E92638
:1042D000000EEA22EF500C6E2C0E0C5C000112E076
:1042E00002EE49F001015F51E926000EEA22EFCF0C
:1042F0000CF003EE54F05E510CC0EBFF5E2B5F2B15
:104300000001E0D7F36A03EE54F001015E51F3CFF0
:10431000EBFF0001120002EE49F001015F51E926B6
:10432000000EEA22EF500C6E2C0E0C5CD8A4010E8D
:104330003B6E500E5F5D010ED8B0000E3B160001C3
:1043400004E001015F2B0001E6D701015F2B0001B2
:10435000120001015B9D000163EC3AF018EC24F0BF
:1043600000EEE9F010EE57F0080EE75204E0E6CF59
:10437000EEFFE82EFAD7EF6A610E4D6E010155513E
:104380000001E8A801D04D902DEC39F000EEE9F0E5
:1043900010EE4EF0080EE75204E0E6CFEEFFE82EF6
:1043A000FAD7EF6A2DEC39F04DB03AD001015551F2
:1043B0000001E8A411D0600E4D6E00EEE9F010EEA1
:1043C00060F0080EE75204E0E6CFEEFFE82EFAD7E1
:1043D000EF6A2DEC39F001D013D0010155510001E5
:1043E000E8A60ED000EEE9F010EE69F0080EE752F4
:1043F00004E0E6CFEEFFE82EFAD7EF6A2DEC39F0B5
:10440000610E4D6E00EEE9F010EE72F0080EE7520C
:1044100004E0E6CFEEFFE82EFAD7EF6A2DEC39F094
:10442000030E4A6E58D9F00E4A6E55D10101796BD0
:10443000786B706B710E6F6FFF0E0101785D00017C
:10444000D8B0E8D070C1AAFF6FC1A9FFD4EC02F0C8
:104450004A6E0D0E4A5CD8B4DDD05C0E4A5CD8A41E
:10446000D1D001016F2B000E70235F6B70C1AAFFCA
:104470006FC1A9FFD4EC02F04A6E4A9A550E4A5C0D
:1044800000010EE100EEE9F010EE9CF00A0EE7529A
:1044900004E0E6CFEEFFE82EFAD7EF6ABCD8B1D041
:1044A000560E4A5C0EE100EEE9F010EEA7F00A0E9F
:1044B000E75204E0E6CFEEFFE82EFAD7EF6AABD87A
:1044C000A0D0570E4A5C0EE100EEE9F010EEB2F01B
:1044D0000A0EE75204E0E6CFEEFFE82EFAD7EF6AC5
:1044E0009AD88FD0580E4A5C0EE100EEE9F010EE3B
:1044F000BDF00A0EE75204E0E6CFEEFFE82EFAD751
:10450000EF6A89D87ED05A0E4A5C16E100EEE9F0D7
:10451000020E016E086A1A6A050E196EA3EC00F00D
:104520002E0EEE6E020E016E010E086E380EA1EC1C
:1045300000F0EE6A70D865D0540E4A5C0EE100EED1
:10454000E9F010EE91F00A0EE75204E0E6CFEEFF3C
:10455000E82EFAD7EF6A5FD854D0530E4A5C0EE1CA
:1045600000EEE9F010EE86F00A0EE75204E0E6CF26
:10457000EEFFE82EFAD7EF6A4ED843D0490E4A5CD8
:104580000EE100EEE9F010EE80F0050EE75204E0D7
:10459000E6CFEEFFE82EFAD7EF6A3DD832D0500EC4
:1045A0004A5C0EE100EEE9F010EEC8F00A0EE752A8
:1045B00004E0E6CFEEFFE82EFAD7EF6A2CD821D040
:1045C000460E4A5C0EE100EEE9F010EED3F00A0E62
:1045D000E75204E0E6CFEEFFE82EFAD7EF6A1BD8E9
:1045E00010D0420E4A5C0DE100EEE9F010EE7BF0D7
:1045F000040EE75204E0E6CFEEFFE82EFAD7EF6AAA
:104600000AD801D068D801016F2B000E7023782BD7
:10461000000112D7120000EEE9F001015F51EB50EA
:104620000C6E000E0C52D8A4010E3B6E0A0E5F5D9C
:10463000010ED8B0000E3B1600010BE000EEE9F0D1
:1046400001015F51EB504A6E5F2B782B000143D87C
:10465000E2D7120094988B8801EC3BF07ADE600E72
:104660004A6E39D801015F6B000102EE49F0010189
:104670005F51E926000EEA22EF500C6E0D0E0C5C25
:10468000D8A4010E3B6EC70E5F5D010ED8B0000EC0
:104690003B1600010FE002EE49F001015F51E926EF
:1046A000000EEA22EF504A6E000115D801015F2B7F
:1046B0000001DAD7000E010155BD010E3B6E010E5F
:1046C0009453D8A4000E3B160001D8A4AFDEC1D885
:1046D00094988B981200010155350001D8B092D002
:1046E000F29A476A080E475C1FE201015C8D4AA0FE
:1046F0005C9D00014CD84AB006D0466A01015A8937
:10470000000114D80DD001015A99462A00010ED893
:10471000050E465C05E1466A01015A89000106D88A
:10472000D8904A32472ADEE3F28A1200E86A010191
:104730005ABB010F5AB9010AD8B45A9BD8A45A8B54
:1047400001015A510001E8BA03D097C152FF02D0CB
:1047500098C152FF9EB219D0F76A96C1F6FF880E33
:10476000F6269C0EF722A66AA68E0800F5CF40FF1B
:104770007EA0FED70101962B7E90170E965D00015C
:1047800002E10101966B0001E5D79E921200010142
:104790005C510001E8AC02D0010E4B1A01015C8DA6
:1047A0004BA05C9DD8904C324B325C510001E8BC70
:1047B00001D01200080E4B1A840E4C1A120001018F
:1047C00055350001D8B0120001015E6B01015E5148
:1047D000605D000116E301015A890001A7DF476A05
:1047E000060E475C06E201015A9900019FDF472A45
:1047F000F7E301015A89000199DF01015E2B0001F5
:10480000E5E31200016A020E086E4A5089EC00F0DE
:10481000200E46EC02F00101912B100E915D00017B
:1048200005E10101916B0D0E46EC02F00001120052
:10483000010155350001D8A06DEC20F063EC3AF091
:104840004C684B688FC1BBFFBC6A9E9254C160F13B
:10485000B6D701015535000104E30D0E46EC02F018
:1048600011D0FF0E4C180101906FFF0E4B184A6ECD
:10487000000131DF90C14AF02EDF93C160F19FDF6C
:104880009EA2FED777EF20F00D0E46EC02F0120E3E
:10489000F76E680EF66E3EEC02F0016A086A1A6A5C
:1048A000050E196EA3EC00F02E0E46EC02F0010E80
:1048B000086E380EA1EC00F0120EF76E7C0EF66E4C
:1048C0003EEC02F00D0E46EC02F0130E096E880E5F
:1048D000026E18EC02F0D8A032EF12F0496E120E00
:1048E000F76E860EF66E3EEC02F00D0E46EC02F010
:1048F000630E46EC02F06D0E46EC02F0640E46ECE0
:1049000002F03E0E46EC02F003D86AD8DFD8FCD79E
:10491000130E096E880E026E18EC02F0F9E3496E70
:10492000010156510001E8A203D0495046EC02F0C3
:104930000D0E495C010ED8A4000E3B6E0A0E495CB8
:10494000010ED8A4000E3B12D8A41200010E486E2E
:1049500049C049F2130E096E880E026E18EC02F07F
:1049600036E3496E010156510001E8A203D04950D7
:1049700046EC02F0080E495C04E14852D8A448060F
:10498000E9D70D0E495C010ED8A4000E3B6E0A0E4D
:10499000495C010ED8A4000E3B124828010ED8A491
:1049A000000E3B120AE002EE49F04850E926000EE4
:1049B000EA220D0EEF6E120008D002EE49F04850C8
:1049C000E926000EEA2249C0EFFF482AC3D702EECB
:1049D00049F04850E926000EEA220D0EEF6E120053
:1049E00001015F6B000102EE49F001015F51E92610
:1049F000000EEA22EF500C6E200E0C5CD8A4010EC3
:104A00003B6E02EE49F05F51E926000EEA22EF50BC
:104A10000C6E0D0E0C5CD8A4010E3B16FD0E5F5DF6
:104A2000010ED8B0000E3B160001D8B446D002EEFD
:104A300049F001015F51E926000EEA22EF500C6EA9
:104A4000610E0C5C000ED8B0010E3B6E02EE49F018
:104A50005F51E926000EEA22EF500C6E7B0E0C5CD3
:104A6000000102E3000E01D0010E3B1614E002EE3D
:104A700049F001015F51E926000EEA22EF500E6E67
:104A8000DF0E0E140C6E02EE49F05F51E926000EA7
:104A9000EA220CC0EFFF000102EE49F001015F5174
:104AA000E926000EEA22EFCF0CF000EEE9F05F51AC
:104AB0000CC0EBFF5F2B000195D7F36A00EEE9F025
:104AC00001015F51F3CFEBFF0001120002014951D8
:104AD0000C6E0A0E0C5C010ED8A4000E3B6E495100
:104AE0000C6E0D0E0C5C010ED8A4000E3B120001E2
:104AF000D8A41200120EF76E9A0EF66E00EEE9F0D0
:104B000091EC04F004E1BDEF28F0F3EF27F0120E72
:104B1000F76EA00EF66E00EEE9F091EC04F009E0FD
:104B2000120EF76EA40EF66E00EEE9F091EC04F0B2
:104B300004E197EF2BF0F3EF27F0120EF76EAC0EB7
:104B4000F66E00EEE9F091EC04F009E0120EF76E5B
:104B5000B00EF66E00EEE9F091EC04F003E13BEFED
:104B60002BF041D2120EF76EB60EF66E00EEE9F0A3
:104B700091EC04F009E0120EF76EBA0EF66E00EE3C
:104B8000E9F091EC04F003E154EF2BF02CD2120E7B
:104B9000F76EC20EF66E00EEE9F091EC04F009E05B
:104BA000120EF76EC60EF66E00EEE9F091EC04F010
:104BB00003E1DBEF2BF017D2120EF76ECE0EF66E7E
:104BC00000EEE9F091EC04F009E0120EF76ED40E5D
:104BD000F66E00EEE9F091EC04F003E102EF2DF047
:104BE00002D2120EF76EDC0EF66E00EEE9F091ECDA
:104BF00004F003E14DEF36F0F6D1120EF76EE20E3F
:104C0000F66E00EEE9F091EC04F002E158D2EBD13F
:104C1000120EF76EEA0EF66E00EEE9F091EC04F07B
:104C200003E125EF2AF0DFD1120EF76EF00EF66EDB
:104C300000EEE9F091EC04F003E1CAEF29F0D3D1E2
:104C4000120EF76EF60EF66E00EEE9F091EC04F03F
:104C500003E11DEF36F0C7D1120EF76EFE0EF66EB1
:104C600000EEE9F091EC04F003E1EFEF28F0BBD1A6
:104C7000130EF76E040EF66E00EEE9F091EC04F000
:104C800009E0130EF76E080EF66E00EEE9F091ECF7
:104C900004F003E136EF36F0A6D1130EF76E100ED6
:104CA000F66E00EEE9F091EC04F009E0130EF76EF9
:104CB000140EF66E00EEE9F091EC04F003E12AEF39
:104CC00035F091D1130EF76E1C0EF66E00EEE9F082
:104CD00091EC04F002E1A2D186D1130EF76E220E00
:104CE000F66E00EEE9F091EC04F003E137EF29F005
:104CF0007AD1130EF76E280EF66E00EEE9F091EC05
:104D000004F003E150EF29F06ED1130EF76E300E70
:104D1000F66E00EEE9F091EC04F009E0130EF76E88
:104D2000360EF66E00EEE9F091EC04F003E19BEF35
:104D300029F059D1130EF76E400EF66E00EEE9F031
:104D400091EC04F009E0130EF76E440EF66E00EEDF
:104D5000E9F091EC04F003E1DAEF30F044D1130E06
:104D6000F76E4E0EF66E00EEE9F091EC04F003E102
:104D7000ADEF31F038D1130EF76E540EF66E00EE33
:104D8000E9F091EC04F009E0130EF76E580EF66EA0
:104D900000EEE9F091EC04F003E1E9EF33F023D108
:104DA000130EF76E620EF66E00EEE9F091EC04F071
:104DB00009E0130EF76E680EF66E00EEE9F091EC66
:104DC00004F003E118EF34F00ED1130EF76E6E0EFF
:104DD000F66E00EEE9F091EC04F003E146EF34F0FA
:104DE00002D1130EF76E740EF66E00EEE9F091EC40
:104DF00004F003E168EF34F0F6D0130EF76E7A0E8C
:104E0000F66E00EEE9F091EC04F003E182EF29F098
:104E1000EAD0130EF76E800EF66E00EEE9F091EC1C
:104E200004F002E156D2DFD0130EF76E860EF66E56
:104E300000EEE9F091EC04F009E0130EF76E8C0E31
:104E4000F66E00EEE9F091EC04F003E1C9EF34F006
:104E5000CAD0130EF76E920EF66E00EEE9F091ECEA
:104E600004F009E0130EF76E980EF66E00EEE9F00E
:104E700091EC04F003E196EF34F0B5D0120EF76E2A
:104E80009A0EF66E00EEE9F091EC04F002E175D1B5
:104E9000AAD0130EF76E9E0EF66E00EEE9F091ECBE
:104EA00004F009E0130EF76EA40EF66E00EEE9F0C2
:104EB00091EC04F002E17AD196D0130EF76EAE0EAB
:104EC000F66E00EEE9F091EC04F003E180EF32F0D1
:104ED0008AD0120EF76EDC0EF66E00EEE9F091EC61
:104EE00004F003E14DEF36F07ED0130EF76EB20EF4
:104EF000F66E00EEE9F091EC04F003E159EF35F0C5
:104F000072D0130EF76EB80EF66E00EEE9F091EC6B
:104F100004F002E19ED067D0130EF76EBE0EF66E5F
:104F200000EEE9F091EC04F002E11ED25CD0130E29
:104F3000F76EC40EF66E00EEE9F091EC04F003E1BA
:104F400072EF2AF050D0130EF76ECE0EF66E00EE12
:104F5000E9F091EC04F003E191EF35F044D0130E49
:104F6000F76ED40EF66E00EEE9F091EC04F002E17B
:104F70004CD139D0130EF76EDA0EF66E00EEE9F072
:104F800091EC04F002E15AD12ED0130EF76E100E00
:104F9000F66E00EEE9F091EC04F003E12AEF35F053
:104FA00022D0130EF76EE00EF66E00EEE9F091ECF3
:104FB00004F002E169D017D0130EF76EE60EF66E1C
:104FC00000EEE9F091EC04F003E153EF33F00BD085
:104FD000130EF76EEE0EF66E00EEE9F091EC04F0B3
:104FE000D8B447EF35F0130EF76EF40EF66E3EECC4
:104FF00002F00D0E46EC02F0630E46EC02F06D0E70
:1050000046EC02F0640E46EC02F03E0E46EC02F076
:10501000640E62EC03F074CF60F1120076EC39F0AC
:1050200070EC3AF001015C310001D8B0CBEF39F0FF
:105030000101D8925AB5D882D8B25681D8A25691D9
:10504000AA6A240EA96E5651DBEC02F00001EBEFC8
:1050500039F076EC39F070EC3AF001015C31000186
:10506000D8B0CBEF39F00101D8925AB5D882D8B276
:105070005685D8A25695AA6A240EA96E5651DBEC25
:1050800002F00001EBEF39F076EC39F070EC3AF019
:1050900001015C310001D8B0CBEF39F00101D892A9
:1050A0005AB5D882D8B2568FD8A2569FAA6A240E73
:1050B000A96E5651DBEC02F00001EBEF39F003EC86
:1050C0003AF004010551300A0611071108110001D8
:1050D0000FE004010751081100010FE1040105511F
:1050E000C00A00010AE104010651120A000105E1AB
:1050F000BC0E04013D6F000136D004010551600A69
:1051000006110711081100010FE0040107510811F1
:1051100000010FE104010551800A00010AE10401C8
:105120000651250A000105E1550E04013D6F0001FD
:105130001AD004010551C00A061107110811000117
:105140000BE0040105510711081100010AE10401F7
:1051500006514B0A000105E11E0E04013D6F0001DE
:1051600002D0CBEF39F0AA6A3B0EA96E04013D5183
:10517000DBEC02F00001EBEF39F070EC3AF00101EA
:105180005C310001D8B0CBEF39F00101D8925AB5AB
:10519000D882D8B25683D8A25693AA6A240EA96E92
:1051A0005651DBEC02F00001EBEF39F070EC3AF015
:1051B00001015C310001D8B0CBEF39F00101D89288
:1051C0005AB5D882D8B25687D8A25697AA6A240E62
:1051D000A96E5651DBEC02F00001EBEF39F003EC65
:1051E0003AF005C495F101019553000103E1010E68
:1051F0000101956F0001AA6A2C0EA96E010195515B
:10520000DBEC02F00001EBEF39F070EC3AF0010159
:105210005C310001D8B0CBEF39F00101D8925AB51A
:10522000D882D8B2568DD8A2569DAA6A240EA96EED
:105230005651DBEC02F00001EBEF39F070EC3AF084
:1052400001015C310001D8B0CBEF39F00101D892F7
:105250005AB5D882D8B25689D8A25699AA6A240ECD
:10526000A96E5651DBEC02F00001EBEF39F070EC67
:105270003AF001015C310001D8B0CBEF39F0010107
:10528000D8925AB5D882D8B25781D8A25791AA6A73
:10529000250EA96E5751DBEC02F00001EBEF39F05F
:1052A00070EC3AF001015C310001D8B0CBEF39F07D
:1052B0000101D8925AB5D882D8B25783D8A2579351
:1052C000AA6A250EA96E5751DBEC02F00001EBEF44
:1052D00039F070EC3AF001015C310001D8B0CBEF4D
:1052E00039F00101D8925AB5D882D8B25787D8A2DE
:1052F0005797AA6A250EA96E5751DBEC02F0000100
:10530000EBEF39F070EC3AF001015C310001D8B0FC
:10531000CBEF39F00101D8925AB5D882D8B257856F
:10532000D8A25795AA6A250EA96E5751DBEC02F058
:105330000001EBEF39F070EC3AF001015C31000153
:10534000D8B0CBEF39F00101D8925AB5D882D8B293
:10535000568BD8A2569BAA6A240EA96E5651DBEC36
:1053600002F00001EBEF39F076EC39F0020149511F
:105370000C6E310E0C5C0001D8B450EF45F0020108
:1053800049510C6E320E0C5C0001D8B42BEF46F084
:10539000CBEF39F076EC39F0F0EC24F00201495112
:1053A0000C6E450E0C5C00011AE176EC39F002013E
:1053B00049510C6E0F0E0C140101946FAA6A2A0E4B
:1053C000A96E9451DBEC02F09453000104E1010159
:1053D000559D000102D00101558D00012CD0020124
:1053E00049510C6E4F0E0C5C000123E102014A5141
:1053F0000C6E460E0C5C000104E10101559D00019C
:1054000017D002014A510C6E4E0E0C5C00010EE1E9
:105410000101558D2A0ED2EC02F0946F94530001D5
:1054200003E1050E0101946F000102D0CBEF39F0CA
:1054300002D0CBEF39F0AA6A230EA96E01015551B3
:10544000DBEC02F00001EBEF39F002014E510C6E83
:105450000D0E0C5C0001D8B4120076EC39F002019C
:1054600049510C6E0D0E0C5C00010CE1AA6A710E24
:10547000A96E0D0EDBEC02F00101559B559D5B956D
:10548000000125D001015E6BFB0E01015E5D000194
:105490001AE202EE49F001015E51E926000EEA220D
:1054A000EF50606FAA6A710E5E25A96ED8B0AA2A65
:1054B0006051DBEC02F00D0E605D000104E00101C3
:1054C0005E2B0001E1E30101558B558D5B850001E9
:1054D000AA6A230EA96E01015551DBEC02F000010E
:1054E000EBEF39F00D0E46EC02F0140EF76E0A0EDB
:1054F000F66E3EEC02F00D0E46EC02F0140EF76E66
:10550000180EF66E3EEC02F00D0E46EC02F0140E94
:10551000F76E3C0EF66E3EEC02F00D0E46EC02F01D
:10552000030E166EE80E63EC03F06DEC20F0010143
:10553000966B9E9A000197C152FF9EBA1CD0170E1F
:105540000101965D000113E2F76A96C1F6FF880E2D
:10555000F6269C0EF722A66AA68E0800F5CF40FF1D
:105560007EA0FED77E900101962B0001E8D70101B5
:10557000966B0001E2D7DF0EAE140101606F440E9E
:10558000605D000109E1FF0E0101975D000102E28B
:105590000101972B0001CED7550E0101605D00017E
:1055A00009E1650E0101975D000102E30101970722
:1055B0000001C0D7450E0101605D0001D8B456D08E
:1055C000530E0101605D0001D8A4B4D7AA6A2E0E63
:1055D000A96E01019751DBEC02F097510C0DF3CF4E
:1055E00067F1F4CF68F1396A386A300E376E830E8E
:1055F000366E68C133F067C132F013EC08F004EC8A
:1056000007F035C066F134C065F133C064F132C0D3
:1056100063F166C135F065C134F064C133F063C134
:1056200032F06AEC06F0986FAA6A2F0EA96E9851B4
:10563000DBEC02F09751170DF3CF67F1F4CF68F16F
:10564000396A386A376A840E366E68C133F067C1CA
:1056500032F013EC08F004EC07F06AEC06F08F6F00
:10566000AA6A2B0EA96E8F51DBEC02F0000177ECD9
:1056700020F0EBEF39F070EC3AF001015C31000101
:10568000D8B0CBEF39F00101D8925AB5D882D8B250
:10569000558FD8A2559FAA6A230EA96E5551DBECEF
:1056A00002F00001EBEF39F003EC3AF0040106518F
:1056B0000711081104E1650E055D000106E3040110
:1056C000086B076B066B640E056F000108C414F0CD
:1056D00007C413F006C412F005C411F01C6A1B6A5B
:1056E000010E1A6E800E196E29EC04F014C027F01A
:1056F00013C026F012C025F011C024F0800E24241F
:105700000401056F000E2520066F000E2620076F8E
:10571000000E2720086F06C454F1AA6A260EA96E4F
:1057200001015451DBEC02F00001EBEF39F076ECB3
:1057300039F001015A510001E8A60AD000EEE9F063
:10574000EE6AEE6AEE6AEE6AEE6AEE6AEE6A02D01F
:105750000DEC38F001015E6B070E01015E5D00018A
:1057600018E200EEE9F001015E51EBCF0CF000EE23
:105770004EF05E510CC0EBFFAA6A5EC1A9FF00EEBD
:10578000E9F05E51EB50DBEC02F001015E2B000111
:10579000E3E3E86A01015AB7010E010AD8B4559152
:1057A000D8A45581AA6A230EA96E5551DBEC02F0EC
:1057B0000001EBEF39F00101559355955597559937
:1057C000000176EC39F001015A510001E8A60BD036
:1057D00000EEE9F0EE6AEE6AEE6AEE6AEE6AEE6AF2
:1057E000EE6AEE6A02D00DEC38F001015A51000168
:1057F000E8B6CBEF39F001015E6B070E01015E5D8B
:1058000000011BE200EEE9F001015E51EBCF0CF06C
:1058100000EE57F05E510CC0EBFFAA6A070E5E2542
:10582000A96ED8B0AA2A00EEE9F05E51EB50DBEC8D
:1058300002F001015E2B0001E0E35E6A0101558385
:105840005A310001D8B0BFD00DEC38F001015A51E7
:105850000001E8B6CBEF39F001015A3100012FE227
:1058600001015E6B070E01015E5D00011BE200EEAF
:10587000E9F001015E51EBCF0CF000EE60F05E51FB
:105880000CC0EBFFAA6A0E0E5E25A96ED8B0AA2A3C
:1058900000EEE9F05E51EB50DBEC02F001015E2B13
:1058A0000001E0E3676B0101558500010DEC38F064
:1058B00001015A510001E8B6CBEF39F015D00101D2
:1058C0005E6B070E01015E5D00010EE2AA6A0E0E1C
:1058D00001015E25A96ED8B0AA2A000EDBEC02F009
:1058E00001015E2B0001EDE301015A3100012FE2BD
:1058F00001015E6B070E01015E5D00011BE200EE1F
:10590000E9F001015E51EBCF0CF000EE69F05E5161
:105910000CC0EBFFAA6A150E5E25A96ED8B0AA2AA4
:1059200000EEE9F05E51EB50DBEC02F001015E2B82
:105930000001E0E3706B0101558700010DEC38F0C8
:1059400001015A510001E8B6CBEF39F015D0010141
:105950005E6B070E01015E5D00010EE2AA6A150E84
:1059600001015E25A96ED8B0AA2A000EDBEC02F078
:1059700001015E2B0001EDE301015E6B070E0101E9
:105980005E5D00011BE200EEE9F001015E51EBCF2C
:105990000CF000EE72F05E510CC0EBFFAA6A1C0E18
:1059A0005E25A96ED8B0AA2A00EEE9F05E51EB5050
:1059B000DBEC02F001015E2B0001E0E3796B0101F9
:1059C0005589000115D001015E6B070E01015E5D76
:1059D00000010EE2AA6A1C0E01015E25A96ED8B074
:1059E000AA2A000EDBEC02F001015E2B0001EDE3C0
:1059F000AA6A230EA96E01015551DBEC02F00001E9
:105A0000EBEF39F00D0E46EC02F0140EF76E620E5D
:105A1000F66E3EEC02F00101553100010EE300EE9E
:105A2000E9F010EE4EF0080EE75204E0E6CFEEFF8C
:105A3000E82EFAD7EF6A4AEC39F00D0E46EC02F088
:105A4000140EF76E6A0EF66E3EEC02F0010155512F
:105A50000001E8A262D000EEE9F010EE57F0080E67
:105A6000E75204E0E6CFEEFFE82EFAD7EF6A4AEC01
:105A700039F0010155510001E8A417D0200E46EC81
:105A800002F0560E46EC02F0200E46EC02F000EE5C
:105A9000E9F010EE60F0080EE75204E0E6CFEEFF0A
:105AA000E82EFAD7EF6A4AEC39F0010155510001AE
:105AB000E8A617D0200E46EC02F0560E46EC02F097
:105AC000200E46EC02F000EEE9F010EE69F0080E50
:105AD000E75204E0E6CFEEFFE82EFAD7EF6A4AEC91
:105AE00039F0010155510001E8A817D0200E46EC0D
:105AF00002F0560E46EC02F0200E46EC02F000EEEC
:105B0000E9F010EE72F0080EE75204E0E6CFEEFF87
:105B1000E82EFAD7EF6A4AEC39F00D0E46EC02F0A7
:105B2000140EF76E740EF66E3EEC02F0016A086A0F
:105B3000DFC327F0DEC326F0DDC325F0DCC324F08D
:105B40003BEC01F0200E46EC02F0480E46EC02F071
:105B50007A0E46EC02F00D0E46EC02F0140EF76ED3
:105B6000800EF66E3EEC02F0016A086AE7C327F089
:105B7000E6C326F0E5C325F0E4C324F03BEC01F0D6
:105B8000200E46EC02F0480E46EC02F07A0E46EC8F
:105B900002F00D0E46EC02F0140EF76E960EF66E45
:105BA0003EEC02F0016A086AE3C327F0E2C326F084
:105BB000E1C325F0E0C324F03BEC01F0200E46ECFD
:105BC00002F0480E46EC02F07A0E46EC02F00D0EA2
:105BD00046EC02F0140EF76EA80EF66E3EEC02F0E4
:105BE000016A04013C51A0EC00F0200E46EC02F0EA
:105BF0006D0E46EC02F0570E46EC02F00D0E46EC30
:105C000002F0520E46EC02F0540E46EC02F046EC66
:105C100002F0590E46EC02F0200E46EC02F00101B3
:105C200056350001D8A0AAD04F0E46EC02F04E0E19
:105C300046EC02F00D0E46EC02F0140EF76EB40EB8
:105C4000F66E3EEC02F0016A086AF1C31AF0F0C386
:105C500019F0A3EC00F0200E46EC02F0480E46ECE2
:105C600002F07A0E46EC02F00D0E46EC02F0140E35
:105C7000F76EC00EF66E3EEC02F0016A086AF3C3DE
:105C80001AF0F2C319F0A3EC00F0200E46EC02F07B
:105C9000420E46EC02F0640E46EC02F00D0E46ECAD
:105CA00002F0140EF76EC80EF66E3EEC02F0016ABA
:105CB0000301F451A0EC00F00D0E46EC02F0140EBE
:105CC000F76ED40EF66E3EEC02F0016AF551A0ECD0
:105CD00000F00D0E46EC02F0140EF76EE00EF66EBC
:105CE0003EEC02F0016A086AEDC31AF0ECC319F049
:105CF0009EEC00F0200E46EC02F0480E46EC02F05E
:105D00007A0E46EC02F00D0E46EC02F0140EF76E21
:105D1000F00EF66E3EEC02F0010157510001E8A4CE
:105D200007D04F0E46EC02F04E0E46EC02F008D0C3
:105D30004F0E46EC02F0460E46EC02F046EC02F046
:105D40000D0E46EC02F0140EF76EFC0EF66E3EECF5
:105D500002F0010157510001E8A607D04F0E46ECB2
:105D600002F04E0E46EC02F008D04F0E46EC02F068
:105D7000460E46EC02F046EC02F008D04F0E46EC20
:105D800002F0460E46EC02F046EC02F00D0E46EC38
:105D900002F0430E46EC02F0570E46EC02F0490EBC
:105DA00046EC02F0440E46EC02F0200E46EC02F007
:105DB00001015631000109E24F0E46EC02F0460E99
:105DC00046EC02F046EC02F059D04F0E46EC02F0E1
:105DD0004E0E46EC02F00D0E46EC02F0150EF76E7C
:105DE0000A0EF66E3EEC02F0016A04013651A0EC98
:105DF00000F0200E46EC02F0570E46EC02F0500E7A
:105E000046EC02F04D0E46EC02F00D0E46EC02F0B0
:105E1000150EF76E120EF66E3EEC02F001015731D0
:105E2000000107E34F0E46EC02F04E0E46EC02F086
:105E300008D04F0E46EC02F0460E46EC02F046EC5F
:105E400002F00D0E46EC02F0150EF76E1A0EF66E0D
:105E50003EEC02F0010157510001E8A207D04F0EBD
:105E600046EC02F04E0E46EC02F008D04F0E46EC27
:105E700002F0460E46EC02F046EC02F001015451ED
:105E8000AB0DF3CF67F1F4CF68F10D0E46EC02F0E5
:105E9000150EF76E220EF66E3EEC02F0016A6851A6
:105EA000A0EC00F00D0E46EC02F0150EF76E2C0E75
:105EB000F66E3EEC02F0016A9351A0EC00F00D0E7C
:105EC00046EC02F0150EF76E340EF66E3EEC02F064
:105ED0008D5146EC02F08E5146EC02F02C0ED2ECC5
:105EE00002F0956F0D0E46EC02F0150EF76E3C0EAB
:105EF000F66E3EEC02F0016A9551A0EC00F00D0E3A
:105F000046EC02F0150EF76E460EF66E3EEC02F011
:105F1000553500010DE3580E46EC02F04D0E46ECEF
:105F200002F0490E46EC02F0540E46EC02F008D0A6
:105F30004F0E46EC02F0460E46EC02F046EC02F044
:105F40000D0E46EC02F0450E46EC02F0430E46EC18
:105F500002F0480E46EC02F04F0E46EC02F0200E26
:105F600046EC02F0010156510001E8A207D04F0EA5
:105F700046EC02F04E0E46EC02F008D04F0E46EC16
:105F800002F0460E46EC02F046EC02F00D0E46EC36
:105F900002F0150EF76E4E0EF66E3EEC02F00101A9
:105FA00056510001E8A607D04F0E46EC02F04E0E07
:105FB00046EC02F008D04F0E46EC02F0460E46ECDE
:105FC00002F046EC02F00D0E46EC02F0150EF76EF4
:105FD000560EF66E3EEC02F0010156510001E8A8A3
:105FE00007D04F0E46EC02F04E0E46EC02F008D001
:105FF0004F0E46EC02F0460E46EC02F046EC02F084
:106000000D0E46EC02F0150EF76E5E0EF66E3EECCF
:1060100002F0010156510001E8AA07D04F0E46ECEC
:1060200002F04E0E46EC02F008D04F0E46EC02F0A5
:10603000460E46EC02F046EC02F00D0E46EC02F085
:10604000150EF76E680EF66E3EEC02F00101565129
:106050000001E8A407D04F0E46EC02F04E0E46ECCD
:1060600002F008D04F0E46EC02F0460E46EC02F06D
:1060700046EC02F03B0ED2EC02F004013D6F0D0E37
:1060800046EC02F0150EF76E700EF66E3EEC02F066
:10609000A10E3D5D000106E3150EF76E780EF66E5B
:1060A0003EEC02F04B0E04013D5D000102E2000EE9
:1060B00001D0010E3B6E640E04013D5D010ED8B0AF
:1060C000000E3B16000106E0150EF76E800EF66E10
:1060D0003EEC02F02A0E04013D5D000106E2150EC1
:1060E000F76E880EF66E3EEC02F00D0E46EC02F0F6
:1060F000540E46EC02F0410E46EC02F0490E46EC1E
:1061000002F04C0E46EC02F0200E46EC02F02A0E95
:10611000D2EC02F00101946F55510001E8AC0DD0B2
:10612000150EF76E920EF66E3EEC02F0016A01015A
:106130009451A0EC00F0000108D04F0E46EC02F0A4
:10614000460E46EC02F046EC02F00D0E46EC02F074
:10615000150EF76E9A0EF66E3EEC02F001015551E7
:106160000001E8AA22D00101686B710E676F786B9D
:10617000FB0E0101785D000117E268C1AAFF67C14B
:10618000A9FFD4EC02F00101606F605146EC02F00F
:106190000D0E605D000108E00101672B000E682311
:1061A0000101782B0001E4E303D00D0E46EC02F070
:1061B000EBEF39F003EC3AF008C4DFF307C4DEF389
:1061C00006C4DDF305C4DCF3C00E0301DC5DCB0EB9
:1061D000DD59170EDE59070EDF590001D8B07DD00A
:1061E00001015E6B150E01015E5D000111E202EE20
:1061F00049F001015E51E926000EEA22EF500C6ED3
:106200000D0E0C5C000104E001015E2B0001EAE3CD
:10621000090E01015E5D00010CE202EE49F0010190
:106220005E51E926000EEA22300EEF6E5E2B000171
:10623000EFD70D0E0201526F0301DF6BDE6BDD6BDA
:10624000DC6B01015E6B090E01015E5D0001D8B0DF
:1062500044D0276A266A256A0A0E246E27C014F0E5
:1062600026C013F025C012F024C011F0DFC31CF0CB
:10627000DEC31BF0DDC31AF0DCC319F029EC04F017
:1062800014C027F013C026F012C025F011C024F06E
:1062900002EE49F001015E51E926000EEA22EF50BC
:1062A0000C6E2B6A2A6A296A0CC028F00F0E28147B
:1062B0002B6A2A6A296A286E24240301DC6F29507C
:1062C0002520DD6F2A502620DE6F2B502720DF6F20
:1062D00001015E2B0001D8A0B6D7070E0301DF5DD8
:1062E000000114E311E1170E0301DE5D00010EE36E
:1062F0000BE1CB0E0301DD5D000108E305E1C00EFB
:106300000301DC5D000102E3000E01D0010E3B6ED3
:10631000810E0301DC5DD90EDD599F0EDE59380E6A
:10632000DF59000102E2000E01D0010E3B12D8A499
:10633000CBEF39F0AA6A300EA96E0301DC51DBEC19
:1063400002F0DD51DBEC02F0DE51DBEC02F0DF515C
:10635000DBEC02F00001EBEF39F003EC3AF008C49B
:10636000E7F307C4E6F306C4E5F305C4E4F3C00E9F
:106370000301E45DCB0EE559170EE659070EE75908
:106380000001D8B07DD001015E6B150E01015E5D8C
:10639000000111E202EE49F001015E51E926000E12
:1063A000EA22EF500C6E0D0E0C5C000104E00101BE
:1063B0005E2B0001EAE3090E01015E5D00010CE2C3
:1063C00002EE49F001015E51E926000EEA22300E8C
:1063D000EF6E5E2B0001EFD70D0E0201526F03012D
:1063E000E76BE66BE56BE46B01015E6B090E010187
:1063F0005E5D0001D8B044D0276A266A256A0A0E7D
:10640000246E27C014F026C013F025C012F024C05B
:1064100011F0E7C31CF0E6C31BF0E5C31AF0E4C3B8
:1064200019F029EC04F014C027F013C026F012C0B4
:1064300025F011C024F002EE49F001015E51E92679
:10644000000EEA22EF500C6E2B6A2A6A296A0CC0F1
:1064500028F00F0E28142B6A2A6A296A286E242431
:106460000301E46F29502520E56F2A502620E66FAE
:106470002B502720E76F01015E2B0001D8A0B6D773
:10648000070E0301E75D000114E311E1170E03019C
:10649000E65D00010EE30BE1CB0E0301E55D0001BB
:1064A00008E305E1C00E0301E45D000102E3000E14
:1064B00001D0010E3B6E810E0301E45DD90EE5595A
:1064C0009F0EE659380EE759000102E2000E01D096
:1064D000010E3B12D8A4CBEF39F0AA6A3D0EA96E8B
:1064E0000301E451DBEC02F0E551DBEC02F0E65194
:1064F000DBEC02F0E751DBEC02F00001EBEF39F0EE
:1065000003EC3AF008C4E3F307C4E2F306C4E1F392
:1065100005C4E0F3800E0301E05D960EE159980E8C
:10652000E259000EE3590001D8B07DD001015E6B45
:10653000150E01015E5D000111E202EE49F001015C
:106540005E51E926000EEA22EF500C6E0D0E0C5C37
:10655000000104E001015E2B0001EAE3080E0101E5
:106560005E5D00010CE202EE49F001015E51E92698
:10657000000EEA22300EEF6E5E2B0001EFD70D0EFB
:106580000201526F0301E36BE26BE16BE06B01010F
:106590005E6B090E01015E5D0001D8B044D0276A30
:1065A000266A256A0A0E246E27C014F026C013F04E
:1065B00025C012F024C011F0E3C31CF0E2C31BF0AD
:1065C000E1C31AF0E0C319F029EC04F014C027F07D
:1065D00013C026F012C025F011C024F002EE49F0DD
:1065E00001015E51E926000EEA22EF500C6E2B6A83
:1065F0002A6A296A0CC028F00F0E28142B6A2A6A0E
:10660000296A286E24240301E06F29502520E16FB8
:106610002A502620E26F2B502720E36F01015E2BCA
:106620000001D8A0B6D7000E0301E35D000114E31A
:1066300011E1980E0301E25D00010EE30BE1960EFD
:106640000301E15D000108E305E1800E0301E05D67
:10665000000102E3000E01D0010E3B6EC10E0301EA
:10666000E05D0E0EE159160EE259020EE3590001EB
:1066700002E2000E01D0010E3B12D8A4CBEF39F09C
:10668000AA6A350EA96E0301E051DBEC02F0E1517C
:10669000DBEC02F0E251DBEC02F0E351DBEC02F068
:1066A0000001EBEF39F076EC39F00301ED6BEC6BA8
:1066B00001015A95020149510C6E2D0E0C5C00012E
:1066C00002E101015A8501015E6B01015E51D89022
:1066D0005AB5010F0C6E0D6A0D360C50490FE96E5C
:1066E000020E0D20EA6EEF500C6E0D0E0C5C0001D8
:1066F00038E001015E51D8905AB5010F0C6E0D6A59
:106700000D360C50490FE96E020E0D20EA6EEF5067
:10671000606F256A0A0E246E25C012F02450116E97
:106720000301EC03F3CF24F0F4CF25F01250EC0377
:10673000F35025261150ED03F350252660C128F0B3
:10674000296A28BE29680F0E2816000E291628501F
:106750002424EC6F29502520ED6F01015E2B0001F0
:10676000B4D701015A510001E8A404D00301EC6D33
:10677000E86AED570301EDAF06D0D00EEC5D8A0E4E
:10678000ED59000102E3000E01D0010E3B6E030142
:10679000EDBF0AD0750EED5D07E3000107E1310E94
:1067A0000301EC5D000102E2000E01D0010E3B127C
:1067B0000001D8A4CBEF39F0AA6A390EA96E030103
:1067C000EC51DBEC02F0ED51DBEC02F00001EBEF01
:1067D00039F003EC3AF006C4F1F305C4F0F3030E0C
:1067E0000301F15D000117E305E1E90E0301F05D2E
:1067F000000111E3150EF76EA20EF66E3EEC02F0EC
:106800000D0E46EC02F0030E0301F16F520EF06F15
:106810000001CBEF39F0AA6A410EA96E0301F051D5
:10682000DBEC02F0F151DBEC02F00001EBEF39F0B0
:1068300003EC3AF006C4F3F305C4F2F3030E0301CC
:10684000F35D000116E305E1E90E0301F25D0001CD
:1068500010E3150EF76EBC0EF66E3EEC02F00D0E58
:1068600046EC02F00301F36B640EF26F0001CBEF14
:1068700039F0AA6A430EA96E0301F251DBEC02F073
:10688000F351DBEC02F00001EBEF39F003EC3AF0EE
:1068900005C4F4F3090E0301F45D00010FE3150EC6
:1068A000F76ED40EF66E3EEC02F00D0E46EC02F0E2
:1068B000070E0301F46F0001CBEF39F0AA6A450E11
:1068C000A96E0301F451DBEC02F00001EBEF39F0AB
:1068D00003EC3AF005C4F5F3030E0301F55D000186
:1068E00002E2000E01D0010E3B6E0F0E0301F55DBA
:1068F000D8A4010E3B1600010FE0150EF76EE80E4E
:10690000F66E3EEC02F00D0E46EC02F0020E0301B4
:10691000F56F0001CBEF39F0AA6A460EA96E0301AC
:10692000F551DBEC02F00001EBEF39F003EC3AF04B
:1069300005C436F401015E6B0F0E01015E5D0001BE
:106940001BE202EE49F001015E51E926000EEA2247
:10695000EF50606F0D0E605D00010EE0AA6A3C0E04
:1069600001015E25A96ED8B0AA2A6051DBEC02F0C5
:1069700001015E2B0001E0E3AA6A3C0E01015E25E5
:10698000A96ED8B0AA2AFF0EDBEC02F00001EBEFF3
:1069900039F003EC3AF005C43CF4AA6A340EA96E4F
:1069A00004013C51DBEC02F03C5111EC08F09AEC94
:1069B00004F035C02BF034C02AF033C029F032C0C7
:1069C00028F0356A346A200E336E820E326E2BC088
:1069D00039F02AC038F029C037F028C036F06AEC08
:1069E00007F035C066F134C065F133C064F132C0E0
:1069F00063F166C135F065C134F064C133F063C141
:106A000032F06AEC06F00101606F150E605D000166
:106A100003E3140E0101606F01016051040D1508BC
:106A2000000114E3F86A820EF324F66E1E0EF420C1
:106A3000F76E0900F5CF11F00900F5CF12F009004B
:106A4000F55009007DEC03F011C001F450EC20F08A
:106A5000EBEF39F00D0E46EC02F0150EF76EFC0E62
:106A6000F66E3EEC02F0016A086A1A6A050E196EAB
:106A7000A3EC00F02E0E46EC02F0010E086E380E6C
:106A8000A1EC00F00D0E46EC02F0EBEF39F04F0EEA
:106A900046EC02F04B0E46EC02F00D0E46EC02F016
:106AA000010E166EF40E63EC03F093EC3BF032EF44
:106AB00012F062EC3EF0CBEC3EF0160EF76E0E0ECE
:106AC000F66E3EEC02F0016A2AC427F029C426F0D3
:106AD00028C425F027C424F0020EDDEC00F0560E89
:106AE00046EC02F0200E46EC02F046EC02F0160EE8
:106AF000F76E160EF66E3EEC02F0016A22C427F025
:106B000021C426F020C425F01FC424F0010EDDECC2
:106B100000F0430E46EC02F00D0E46EC02F0EBEFF7
:106B200039F0160EF76E1E0EF66E3EEC02F00D0EEC
:106B300046EC02F0939A8A8A32EC20F08BEC20F03B
:106B40000B0E096EB80E026E18EC02F0F9E30101AB
:106B5000606F440E605D010ED8A4000E3B6E640EA3
:106B6000605D010ED8A4000E3B12000114E0040188
:106B700001510001E8BE06D004010153000102E00A
:106B8000040101070001016A04010151A0EC00F0B9
:106B90000D0E46EC02F0550E0101605D010ED8A409
:106BA000000E3B6E750E605D010ED8A4000E3B1208
:106BB000000112E0040101BF04D07F0E015D00015D
:106BC00002E20401012B0001016A04010151A0EC61
:106BD00000F00D0E46EC02F0450E0101605D010E65
:106BE000D8A4000E3B6E650E605D010ED8A4000EA9
:106BF0003B12000104E077EC20F0EBEF39F0530E8C
:106C00000101605D010ED8A4000E3B6E730E605D45
:106C1000010ED8A4000E3B1200010CE077EC20F02E
:106C2000AA6A340EA96E04010151DBEC02F00001E6
:106C3000EBEF39F050EC20F083D776EC39F002011D
:106C4000495101018D6F02014A5101018E6FAA6AFB
:106C5000280EA96E8D51DBEC02F0AA6A290EA96EEE
:106C60008E51DBEC02F00001EBEF39F003EC3AF06F
:106C700005C493F1020E0101935D000103E2020ECF
:106C80000101936F0001AA6A2D0EA96E01019351B3
:106C9000DBEC02F00001EBEF39F00D0E46EC02F0F8
:106CA000160EF76E420EF66E3EEC02F00D0E46EC3E
:106CB00002F00D0E46EC02F0160EF76E5C0EF66E4C
:106CC0003EEC02F00D0E46EC02F0160EF76E7C0E56
:106CD000F66E3EEC02F00D0E46EC02F0160EF76E6C
:106CE0009A0EF66E3EEC02F00D0E46EC02F0160E19
:106CF000F76EC40EF66E3EEC02F00D0E46EC02F09E
:106D0000160EF76EEE0EF66E3EEC02F00D0E46EC31
:106D100002F0170EF76E140EF66E3EEC02F00D0E3A
:106D200046EC02F0170EF76E480EF66E3EEC02F0DF
:106D30000D0E46EC02F0170EF76E7E0EF66E3EEC70
:106D400002F00D0E46EC02F0170EF76E9A0EF66E7C
:106D50003EEC02F00D0E46EC02F0170EF76EC00E80
:106D6000F66E3EEC02F00D0E46EC02F0170EF76EDA
:106D7000D60EF66E3EEC02F00D0E46EC02F0180E4A
:106D8000F76E0E0EF66E3EEC02F00D0E46EC02F0C3
:106D9000180EF76E2A0EF66E3EEC02F00D0E46EC63
:106DA00002F0180EF76E560EF66E3EEC02F00D0E67
:106DB00046EC02F0180EF76E760EF66E3EEC02F020
:106DC0000D0E46EC02F0180EF76E9E0EF66E3EECBF
:106DD00002F00D0E46EC02F0180EF76ECA0EF66EBB
:106DE0003EEC02F00D0E46EC02F0180EF76EFA0EB5
:106DF000F66E3EEC02F00D0E46EC02F0190EF76E48
:106E00001E0EF66E3EEC02F00D0E46EC02F0190E70
:106E1000F76E640EF66E3EEC02F00D0E46EC02F0DC
:106E2000190EF76E8A0EF66E3EEC02F00D0E46EC71
:106E300002F0190EF76EBE0EF66E3EEC02F00D0E6D
:106E400046EC02F0190EF76EE40EF66E3EEC02F020
:106E50000D0E46EC02F01A0EF76E0E0EF66E3EECBC
:106E600002F00D0E46EC02F01A0EF76E400EF66EB2
:106E70003EEC02F00D0E46EC02F01A0EF76E700EAC
:106E8000F66E3EEC02F00D0E46EC02F01A0EF76EB6
:106E90009E0EF66E3EEC02F00D0E46EC02F01A0E5F
:106EA000F76ECC0EF66E3EEC02F00D0E46EC02F0E4
:106EB0001A0EF76EE20EF66E3EEC02F00D0E46EC88
:106EC00002F01B0EF76E120EF66E3EEC02F00D0E87
:106ED00046EC02F01B0EF76E500EF66E3EEC02F022
:106EE0000D0E46EC02F01B0EF76E6E0EF66E3EECCB
:106EF00002F00D0E46EC02F01B0EF76E980EF66EC9
:106F00003EEC02F00D0E46EC02F01B0EF76EB60ED4
:106F1000F66E3EEC02F00D0E46EC02F01B0EF76E24
:106F2000DE0EF66E3EEC02F00D0E46EC02F01C0E8C
:106F3000F76E2A0EF66E3EEC02F00D0E46EC02F0F5
:106F40001C0EF76E500EF66E3EEC02F00D0E46EC87
:106F500002F01C0EF76E640EF66E3EEC02F00D0EA3
:106F600046EC02F01C0EF76E840EF66E3EEC02F05C
:106F70000D0E46EC02F01C0EF76EA40EF66E3EEC03
:106F800002F00D0E46EC02F01C0EF76EC40EF66E0B
:106F90003EEC02F00D0E46EC02F01C0EF76EE40E15
:106FA000F66E3EEC02F00D0E46EC02F01D0EF76E92
:106FB0000A0EF66E3EEC02F00D0E46EC02F01D0ECF
:106FC000F76E300EF66E3EEC02F00D0E46EC02F05F
:106FD0001D0EF76E580EF66E3EEC02F00D0E46ECEE
:106FE00002F01D0EF76E720EF66E3EEC02F00D0E04
:106FF00046EC02F01D0EF76EA40EF66E3EEC02F0AB
:107000000D0E46EC02F01D0EF76ED40EF66E3EEC41
:1070100002F00D0E46EC02F0DED101015A9700019C
:10702000F0EC24F001015A915E6B000102EE49F090
:1070300001015E51E926000EEA22EF500C6E2D0E82
:107040000C5CD8A4010E3B6E02EE49F05E51E926BD
:10705000000EEA22EF500C6E200E0C5CD8A4010E3C
:107060003B1602EE49F05E51E926000EEA22EF508F
:107070000C6E0D0E0C5CD8A4010E3B160A0E5E5D64
:10708000010ED8B0000E3B16000111E002EE49F0EF
:1070900001015E51E926000EEA22EFCF0CF000EE6E
:1070A000E9F05E510CC0EBFF5E2B0001BED7060E6F
:1070B00001015E5D000112E25EC15FF1060E010199
:1070C0005F5D00010BE2200EF36E00EEE9F00101BE
:1070D0005F51F3CFEBFF5F2B0001F0D702EE49F0D9
:1070E00001015E51E926000EEA22EF500C6E200EDF
:1070F0000C5C0001D8B4EF6B02EE49F001015E5167
:10710000E926000EEA22EF500C6E0D0E0C5C000119
:1071100005E101015A810001EF6B120002EE49F016
:1071200001015E51E926000EEA22EF500C6E2D0E91
:107130000C5C0001D8A46AD001015E2B02EE49F07C
:107140005E51E926000EEA22EF500C6E0F0E0C1471
:107150004D6E5E2B02EE49F05E51E926000EEA22EA
:10716000EF500C6E300E0C5C000ED8B0010E3B6E72
:1071700002EE49F05E51E926000EEA22EF500C6E55
:107180003A0E0C5C000102E3000E01D0010E3B162A
:1071900029E0256A0A0E246E25C011F04D50240204
:1071A000F3CF24F0F4CF25F01102F350252602EEA0
:1071B00049F001015E51E926000EEA22EF500C6E03
:1071C000296A0CC028F00F0E2816000E291624502C
:1071D00028244D6E100E4D5C000102E30F0E4D6E23
:1071E00001015E2B00014DC0EFF002EE49F00101FC
:1071F0005E51E926000EEA22EF500C6E0D0E0C5C7B
:10720000000104E101015A810001120001015E2B1D
:1072100002EE49F05E51E926000EEA22EF500C6EB4
:10722000560E0C5C010ED8A4000E3B6E02EE49F027
:107230005E51E926000EEA22EF500C6E760E0C5CD1
:10724000010ED8A4000E3B12000103E04FD84ED827
:1072500002D001015A870001120001015E6B070E86
:1072600001015E5D000115E200EEE9F001015E51F1
:10727000EB500C6ED8900C344A6E060E5E5D000129
:1072800002E14D504A126BEC23F001015E2B00012C
:10729000E6E3120001015E6B000100EEE9F001017E
:1072A0005E51EB500C6E200E0C5CD8A4010E3B6EB0
:1072B000060E5E5D010ED8B0000E3B1600010AE01E
:1072C00000EEE9F001015E51EB5046EC02F05E2B5E
:1072D0000001E2D7EF510C6E0C5207E02D0E46EC88
:1072E00002F0016AEF51A0EC00F0120001015A9780
:1072F000786B000102EE49F001017851E926000E99
:10730000EA22EF500C6E200E0C5CD8A4010E3B6EEE
:10731000FD0E785D010ED8B0000E3B16000115E0A1
:1073200002EE49F001017851E926000EEA22EF5001
:107330000C6E0D0E0C5C000104E101015A87000186
:1073400012000101782B0001D4D70101782B78516C
:10735000FF080B6E5F6B01015F510B5C00011AE3CC
:1073600001015F5178250E6E0F6A0F360E50490FDE
:10737000E96E020E0F20EA6EEFCF0CF002EE49F03C
:107380005F51E926000EEA220CC0EFFF01015F2BDE
:107390000001E1E31200450E46EC02F0520E46EC0D
:1073A00002F046EC02F04F0E46EC02F0520E46ECB4
:1073B00002F00D0E46EC02F0630E46EC02F06D0E8C
:1073C00046EC02F0640E46EC02F03E0E46EC02F093
:1073D000AECF60F112004F0E46EC02F04B0E46ECC1
:1073E00002F00D0E46EC02F0630E46EC02F06D0E5C
:1073F00046EC02F0640E46EC02F03E0E46EC02F063
:10740000AECF60F1120072DF010E01015E6F02016A
:1074100049510C6E0F0B0401086B076B066B056F6F
:10742000000102EE49F001015E51E926000EEA2258
:10743000EF500C6E0D0E0C5C0001D8B443D0276ADF
:10744000266A256A0A0E246E27C014F026C013F09F
:1074500025C012F024C011F008C41CF007C41BF0B2
:1074600006C41AF005C419F029EC04F014C027F082
:1074700013C026F012C025F011C024F002EE49F02E
:1074800001015E51E926000EEA22EF500C6E2B6AD4
:107490002A6A296A0CC028F00F0E28142B6A2A6A5F
:1074A000296A286E24240401056F29502520066FBF
:1074B0002A502620076F2B502720086F01015E2BD2
:1074C0000001AED71200466A476A486A4A6A4C6AA7
:1074D0004B6A4D6A0101916B5A8B966B0001120049
:1074E00005DFF0EC24F001015C91020149510C6EC2
:1074F0004F0E0C5C010ED8A4000E3B6E4A510C6E70
:107500004E0E0C5C010ED8A4000E3B16000104E0E8
:1075100001015A85000158D0020149510C6E590EE3
:107520000C5C010ED8A4000E3B6E4A510C6E450E49
:107530000C5C010ED8A4000E3B164B510C6E530E82
:107540000C5C010ED8A4000E3B16000104E0010102
:107550005A85000139D0020149510C6E4F0E0C5C66
:10756000010ED8A4000E3B6E4A510C6E460E0C5C08
:10757000010ED8A4000E3B164B510C6E460E0C5C4F
:10758000010ED8A4000E3B16000104E001015A953B
:1075900000011AD0020149510C6E4E0E0C5C010E16
:1075A000D8A4000E3B6E4A510C6E4F0E0C5C010EBF
:1075B000D8A4000E3B16000104E001015A95000119
:1075C00002D001015C810001120001015E6B070E17
:1075D00001015E5D000113E201015E516725A96EA4
:1075E000000E6821AA6ED4EC02F00C6E00EEE9F0F9
:1075F0005E510CC0EBFF01015E2B0001E8E3F06B74
:107600001200010155510001E8AA8CD001015F6B05
:10761000926B5C975C9BFA0E01015F5D0001D8B034
:1076200081D0AA6A710E01015F25A96ED8B0AA2A7D
:10763000D4EC02F0606F0D0E605D0001D8B472D022
:107640005C0E0101605D0001D8A468D001015C8777
:107650005F2BAA6A710E5F25A96ED8B0AA2AD4EC56
:1076600002F0606F609B550E605D0001D8B473EC52
:1076700044F0560E0101605D010ED8A4000E3B6E71
:10768000570E605D010ED8A4000E3B120001D8A475
:107690002EEC3FF0540E0101605D0001D8B4C3EC44
:1076A00043F0580E0101605D0001D8B41BEC44F0BA
:1076B000420E0101605D00010CE100EE7BF013EE73
:1076C0004EF0050EE75204E0E6CFEEFFE82EFAD7C3
:1076D000EF6A010156510001E8A619D0530E0101CD
:1076E000605D010ED8A4000E3B6E490E605D010E78
:1076F000D8A4000E3B12000103E0E2EC44F007D0F6
:10770000530E0101605D0001D8B4B2EC44F00101F8
:1077100056510001E8AA02D0B2EC4EF001015F2BF5
:10772000000179D71200230ED2EC02F00101556F4F
:10773000240ED2EC02F0566F250ED2EC02F0576FF9
:10774000260ED2EC02F0546F0001BDDE2B0ED2ECFF
:1077500002F001018F6F2E0ED2EC02F0976F2F0E08
:10776000D2EC02F0986FCD80280ED2EC02F08D6F33
:10777000290ED2EC02F08E6F2D0ED2EC02F0936F38
:10778000946B010E956F5531000111E30101686B97
:10779000676B00011ADF00EE4EF010EEE9F0230EE9
:1077A000E75204E0E6CFEEFFE82EFAD7EF6A0101D8
:1077B00055510001E8A212D00101686B070E676FF6
:1077C000000103DF00EE57F010EEE9F0230EE75260
:1077D00004E0E6CFEEFFE82EFAD7EF6A010155513B
:1077E0000001E8A412D00101686B0E0E676F000162
:1077F000ECDE00EE60F010EEE9F0230EE75204E05C
:10780000E6CFEEFFE82EFAD7EF6A010155510001ED
:10781000E8A612D00101686B150E676F0001D5DE76
:1078200000EE69F010EEE9F0230EE75204E0E6CF37
:10783000EEFFE82EFAD7EF6A010155510001E8A8E2
:1078400012D00101686B1C0E676F0001BEDE00EEF6
:1078500072F010EEE9F0230EE75204E0E6CFEEFFFF
:10786000E82EFAD7EF6A300ED2EC02F00301DC6F9B
:10787000D4EC02F0DD6FD4EC02F0DE6FD4EC02F059
:10788000DF6F070EDF5D000114E311E1170E030146
:10789000DE5D00010EE30BE1CB0E0301DD5D0001B7
:1078A00008E305E1C00E0301DC5D000102E3000E08
:1078B00001D0010E3B6E810E0301DC5DD90EDD5956
:1078C0009F0EDE59380EDF59000102E2000E01D092
:1078D000010E3B1208E0080E0301DF6FA10EDE6F00
:1078E000790EDD6FDC6B00013D0ED2EC02F003017E
:1078F000E46FD4EC02F0E56FD4EC02F0E66FD4EC68
:1079000002F0E76F070EE75D000114E311E1170EC7
:107910000301E65D00010EE30BE1CB0E0301E55D23
:10792000000108E305E1C00E0301E45D000102E38C
:10793000000E01D0010E3B6E810E0301E45DD90EF5
:10794000E5599F0EE659380EE759000102E2000E94
:1079500001D0010E3B1209E0080E0301E76F990EFA
:10796000E66F140EE56F900EE46F960E0401356F0E
:10797000340ED2EC02F03C6F3C5111EC08F09AEC62
:1079800004F035C02BF034C02AF033C029F032C0E7
:1079900028F0356A346A200E336E820E326E2BC0A8
:1079A00039F02AC038F029C037F028C036F06AEC28
:1079B00007F035C066F134C065F133C064F132C000
:1079C00063F166C135F065C134F064C133F063C161
:1079D00032F06AEC06F00101606F150E605D000187
:1079E00003E3140E0101606F01016051040D1508DD
:1079F000000114E3F86ADA0EF324F66E1E0EF4208A
:107A0000F76E0900F5CF11F00900F5CF12F009006B
:107A1000F55009007DEC03F011C001F4030E0101E3
:107A20006027150E605D000103E3140E0101606F15
:107A300001016051040D1508000114E3F86A320ECB
:107A4000F324F66E1F0EF420F76E0900F5CF11F047
:107A50000900F5CF12F00900F55009007DEC03F0A4
:107A600011C037F4140E0401316F3C0ED2EC02F059
:107A7000366F140E365D000103E2140E0401366FFA
:107A8000790E0401365D000103E3780E0401366FC0
:107A90000001040E126EB00E116E166A36C415F097
:107AA000D7EC03F00401316F350ED2EC02F0030184
:107AB000E06FD4EC02F0E16FD4EC02F0E26FD4ECB2
:107AC00002F0E36F000EE35D000114E311E1980E94
:107AD0000301E25D00010EE30BE1960E0301E15D9F
:107AE000000108E305E1800E0301E05D000102E30F
:107AF000000E01D0010E3B6E410E0301E05D8A0EC7
:107B0000E159F70EE259010EE359000102E2000EBD
:107B100001D0010E3B1209E0010E0301E36FC90E13
:107B2000E26FC30EE16F800EE06F0001390ED2EC00
:107B300002F00301EC6FD4EC02F0ED6FEDAF06D074
:107B4000D00EEC5D8A0EED59000102E3000E01D06B
:107B5000010E3B6E0301EDBF0AD0750EED5D07E32C
:107B6000000107E1310E0301EC5D000102E2000EAD
:107B700001D0010E3B12000105E0040E0301ED6F80
:107B80004C0EEC6F00013B0ED2EC02F004013D6F95
:107B9000410ED2EC02F00301F06FD4EC02F0F16F71
:107BA000030EF15D00010BE305E1E90E0301F05D59
:107BB000000105E3030E0301F16F520EF06F0001A7
:107BC000430ED2EC02F00301F26FD4EC02F0F36F3B
:107BD000030EF35D00010AE305E1E90E0301F25D26
:107BE000000104E30301F36B640EF26F0001450E24
:107BF000D2EC02F00301F46F090EF45D000103E31F
:107C0000070E0301F46F0001460ED2EC02F00301EF
:107C1000F56F030EF55D000102E2000E01D0010ECA
:107C20003B6E0F0E0301F55DD8A4010E3B1600015B
:107C300003E0020E0301F56F300E0301C96F03EE7E
:107C40004EF0EF6A04013B6B01EE3DF0EE6E2E0E3E
:107C5000EE6E300EEE6EEF6A03014B6B4A6B4D6BAE
:107C60004C6B146A0F0E136E420E126E400E116EA4
:107C7000F2C319F0F3C31AF01B6A1C6AA9EC03F0F3
:107C800012C00CF411C00BF40F0EF55D00010DE0F5
:107C90000301F55104010B03F3CF0DF4F4CF0EF4FF
:107CA0000C03F3500E2700010BD0D89004010C31C7
:107CB000256E0B31246E0B250D6F25500C210E6F98
:107CC000000112008194949E8B9E810E026E010E23
:107CD000096E810E036E040E046E010E0A6E116EA3
:107CE0002CEC03F0949E8B8E81A6FED7949E8B9EE7
:107CF000810E026E010E096E810E036E040E046E7B
:107D0000010E0A6E440E116E2CEC03F0810E026E11
:107D1000020E096E810E036E040E046E0A6A00ECF8
:107D200003F011C060F101016029000108E0949E98
:107D30008B8E010E62EC03F0949E8B9ED9D7810E40
:107D4000026E020E096E810E036E040E046E0A6A44
:107D500000EC03F011C03EF400EC03F011C03FF45E
:107D600000EC03F011C040F400EC03F011C041F44A
:107D700000EC03F011C042F400EC03F011C043F436
:107D800000EC03F011C044F400EC03F011C045F422
:107D9000949E8B8E12001D0EF76EF20EF66E3EEC68
:107DA00002F0016A04013E51A0EC00F00D0E46EC19
:107DB00002F01E0EF76E020EF66E3EEC02F0016A45
:107DC000020E086E3F5189EC00F0020E086E405121
:107DD00089EC00F00D0E46EC02F01E0EF76E0C0E54
:107DE000F66E3EEC02F0016A020E086E415189EC1B
:107DF00000F00D0E46EC02F01E0EF76E1C0EF66E35
:107E00003EEC02F0016A020E086E425189EC00F06D
:107E1000020E086E435189EC00F00D0E46EC02F0A4
:107E20001E0EF76E300EF66E3EEC02F0016A020E88
:107E3000086E445189EC00F00D0E46EC02F01E0E67
:107E4000F76E400EF66E3EEC02F0016A020E086E0E
:107E5000455189EC00F00D0E46EC02F0030E0301D3
:107E6000876F140E886F180E896F8A6B060E8B6FE2
:107E700000016DEC43F0030189510101686F0301BA
:107E80008A510101676F67C132F068C133F013ECAA
:107E900008F0396A386A400E376E800E366E6AEC2A
:107EA00007F035C027F034C026F033C025F032C0CB
:107EB00024F0396A386A200E376E890E366E27C074
:107EC00035F026C034F025C033F024C032F004EC85
:107ED00007F035C02AF434C029F433C028F432C086
:107EE00027F400EEA7F0020E016E2AC427F029C481
:107EF00026F028C425F027C424F0DDEC00F0EF6A5A
:107F000003018B510101686F03018C510101676FFF
:107F1000340E666F330E656F630E646F7C0E636F95
:107F200067C132F068C133F013EC08F066C139F074
:107F300065C138F064C137F063C136F06AEC07F010
:107F400035C027F034C026F033C025F032C024F00D
:107F5000396A800E386E140E376E870E366E27C063
:107F600035F026C034F025C033F024C032F074EC74
:107F700006F035C022F434C021F433C020F432C0FE
:107F80001FF400EEB2F0020E016E22C427F021C4ED
:107F900026F020C425F01FC424F0010EDDEC00F013
:107FA000EF6A0001120001015F6B00015EEC21F03D
:107FB000256A0A0E246E030154510C6E296A0CC006
:107FC00028F00F0E2816000E291625C01AF024508E
:107FD000196E2802F3CF24F0F4CF25F01A502802AE
:107FE000F350252619502902F350252655510E6EBF
:107FF000296A0EC028F00F0E2816000E29162450EC
:10800000282404014E6F256A0A0E246E030156517E
:108010000C6E296A0CC028F00F0E2816000E2916C7
:1080200025C01AF02450196E2802F3CF24F0F4CFA3
:1080300025F01A502802F350252619502902F35032
:10804000252657510E6E296A0EC028F00F0E2816ED
:10805000000E29162450282404014F6F396A386A0B
:10806000700E376E840E366E4F5111EC08F004EC32
:1080700007F035C027F034C026F033C025F032C0F9
:1080800024F04E5111EC08F027C039F026C038F02A
:1080900025C037F024C036F076EC06F035C066F126
:1080A00034C065F133C064F132C063F1256A0A0E51
:1080B000246E030159510C6E296A0CC028F00F0E72
:1080C0002816000E291625C01AF02450196E280211
:1080D000F3CF24F0F4CF25F01A502802F3502526D0
:1080E00019502902F35025265A510E6E296A0EC0E6
:1080F00028F00F0E2816000E2916245028240401FB
:10810000536F01015F6B00015DEC21F003EE54F051
:10811000EECFF3FFEFCFF4FFF3504E0AF41005E17A
:108120005A0E04014E27000115D004014E515A0881
:108130004E6F4F5300010EE004014E074F513C08B3
:108140004F6F5353000105E004014F07535164087A
:10815000536F0001D89004014F37D8905337010175
:108160005F6B00015CEC21F0256A640E246E030154
:1081700054510C6E296A0CC028F00F0E2816000E00
:10818000291625C01AF02450196E2802F3CF24F0C6
:10819000F4CF25F01A502802F35025261950290251
:1081A000F3502526296A0A0E286E55510E6E2D6A47
:1081B0000EC02CF00F0E2C16000E2D1629C01AF032
:1081C0002850196E2C02F3CF28F0F4CF29F01A5062
:1081D0002C02F350292619502D02F350292628503D
:1081E0002426295025225651106E296A10C028F0E5
:1081F0000F0E2816000E2916285024240401506F53
:1082000029502520516F256A0A0E246E030157510B
:108210000C6E296A0CC028F00F0E2816000E2916C5
:1082200025C01AF02450196E2802F3CF24F0F4CFA1
:1082300025F01A502802F350252619502902F35030
:10824000252658510E6E296A0EC028F00F0E2816EA
:10825000000E2916245028240401526F396A386A06
:10826000700E376E840E366E525111EC08F004EC2D
:1082700007F035C027F034C026F033C025F032C0F7
:1082800024F050C432F051C433F013EC08F027C08E
:1082900039F026C038F025C037F024C036F076EC2F
:1082A00006F035C066F134C065F133C064F132C008
:1082B00063F1256A0A0E246E03015A510C6E296A75
:1082C0000CC028F00F0E2816000E291625C01AF033
:1082D0002450196E2802F3CF24F0F4CF25F01A5061
:1082E0002802F350252619502902F35025265B5108
:1082F0000E6E296A0EC028F00F0E2816000E2916E1
:10830000245028240401546F01015F6B00015BECD1
:1083100021F003EE54F0EECFF3FFEFCFF4FFF35074
:10832000450AF41007E1B40E04015027000E512352
:1083300000011AD004015051B408506F000E51557D
:10834000516F5253000110E004015007000E515BC1
:1083500052513C08526F5453000105E0040152078A
:1083600054516408546F000103EE54F0EF6A51C495
:1083700012F050C411F0166A140E156ED7EC03F00B
:10838000246E12C025F0410E24240101606F03EE1B
:1083900054F0EE50FEE1ED5260C1EEFFEF6A4EC4C4
:1083A00011F00A0ED4EC03F0246E256A410E242449
:1083B000606F03EE54F0EE50FEE1ED5260C1EEFF4F
:1083C000EF6A256A300E246E51C429F050C428F09B
:1083D00029C012F028C011F0166A140E156ED7ECE1
:1083E00003F01AC029F019C028F0D8902932283299
:1083F00024502824606F03EE54F0EE50FEE1ED525D
:1084000060C1EEFFEF6A126A4EC411F0166A0A0EDE
:10841000156ED7EC03F01AC025F019C024F0300E09
:108420002424606F03EE54F0EE50FEE1ED5260C183
:10843000EEFFEF6A256A410E246E000E040150B172
:10844000010E296A286E29503C0DF3CF29F02850DF
:108450003C0DF3CF28F0F450292652512826000E67
:10846000292229C012F028C011F0166A050E156ED7
:10847000D7EC03F0286E12C029F024502824010103
:10848000606F03EE54F0EE50FEE1ED5260C1EEFF7E
:10849000EF6A4FC411F0050ED4EC03F0246E256A88
:1084A000410E2424606F03EE54F0EE50FEE1ED52D5
:1084B00060C1EEFFEF6A3C0E040150A1000E246E75
:1084C00050A1000E256E525124240101676F000E49
:1084D0002520686F68C112F067C111F0166A050E99
:1084E000156ED7EC03F019C060F16051640DF3CF45
:1084F00024F0F4CF25F00401545124240101676FC6
:10850000000E2520686F68C112F067C111F0166A6D
:10851000320E156ED7EC03F0246E12C025F0300E2B
:108520002424606F03EE54F0EE50FEE1ED5260C182
:10853000EEFFEF6A68C112F067C111F0166A320EE1
:10854000156ED7EC03F019C054F4126A4FC411F041
:10855000166A050E156ED7EC03F019C060F1605174
:10856000640DF3CF24F0F4CF25F0040153512424FB
:108570000101676F000E2520686F68C112F067C1A6
:1085800011F0166A320E156ED7EC03F0246E12C08D
:1085900025F0300E2424606F68C112F067C111F01D
:1085A000166A320E156ED7EC03F019C053F403EEC1
:1085B00054F0EE50FEE1ED5260C1EEFFEF6ADF0EC7
:1085C000396E4F0E386E050E376E800E366E040112
:1085D000545111EC08F004EC07F035C027F034C01A
:1085E00026F033C025F032C024F0356A346A020E1A
:1085F000336E850E326E27C039F026C038F025C0A4
:1086000037F024C036F076EC06F0B8EC07F0010144
:10861000606F03EE54F0EE50FEE1ED5260C1EEFFEC
:10862000EF6ADF0E396E4F0E386E050E376E800E14
:10863000366E0401535111EC08F004EC07F035C01C
:1086400027F034C026F033C025F032C024F0356A5C
:10865000346A020E336E850E326E27C039F026C0A2
:1086600038F025C037F024C036F076EC06F0B8ECD0
:1086700007F00101606F03EE54F0EE50FEE1ED52A1
:1086800060C1EEFFEF6A0001120081A6FED7949E42
:108690008B9E030187510B6E010E0401556F04017F
:1086A00055510B5C000116E3810E026E010E096E3E
:1086B000810E036E040E046E010E0A6E03EE87F047
:1086C00004015551EB50116E2CEC03F00401552BB5
:1086D0000001E5E3949E8B8E12008194D6DF81A683
:1086E000FED7949E8B9E810E026E010E096E810E46
:1086F000036E040E046E010E0A6E440E116E2CEC15
:1087000003F0810E026E020E096E810E036E040EDE
:10871000046E0A6A00EC03F011C060F101016029E7
:10872000000108E0949E8B8E010E62EC03F0949E93
:108730008B9ED9D703EE87F004015551EB500C6E98
:108740000C040101606F0401556B040155510101D6
:10875000605D000115E3810E026E020E096E810E4E
:10876000036E040E046E0A6A00EC03F003EE87F059
:108770000401555111C0EBFF0401552B0001E5E345
:10878000949E8B8E120001016A6B696B5E6B0A0E00
:1087900001015E5D00010FE2010EEAEC02F00C6ED9
:1087A00025C00DF00C50010169270D506A2301010D
:1087B0005E2B0001ECE369C132F06AC133F013ECC7
:1087C00008F0396A400E386E1C0E376E8A0E366E0F
:1087D00074EC06F035C027F034C026F033C025F025
:1087E00032C024F0396A386A480E376E840E366E0D
:1087F00027C035F026C034F025C033F024C032F055
:1088000004EC07F035C01EF434C01DF433C01CF472
:1088100032C01BF400EE91F0020E016E1EC427F070
:108820001DC426F01CC425F01BC424F0010EDDEC91
:1088300000F0EF6A12000101686B676B5E6B0A0E55
:1088400001015E5D00010FE2000EEAEC02F00C6E29
:1088500025C00DF00C50010167270D506823010160
:108860005E2B0001ECE367C132F068C133F013EC1A
:1088700008F0396A400E386E1C0E376E8A0E366E5E
:1088800074EC06F035C027F034C026F033C025F074
:1088900032C024F0396A386A480E376E840E366E5C
:1088A00027C035F026C034F025C033F024C032F0A4
:1088B00004EC07F035C026F434C025F433C024F4AA
:1088C00032C023F400EEBDF0020E016E26C427F084
:1088D00025C426F024C425F023C424F0010EDDECC9
:1088E00000F0EF6A12000101686B676B5E6B0A0EA5
:1088F00001015E5D00010FE2030EEAEC02F00C6E76
:1089000025C00DF00C50010167270D5068230101AF
:108910005E2B0001ECE3396A400E386E1C0E376E98
:108920008B0E366E68C133F067C132F013EC08F07D
:1089300004EC07F035C014F434C013F433C012F45F
:1089400032C011F400EE9CF0020E016E14C427F048
:1089500013C426F012C425F011C424F0DDEC00F09D
:10896000EF6A12000101686B676B5E6B0A0E010112
:108970005E5D00010FE20F0EEAEC02F00C6E25C006
:108980000DF00C50010167270D50682301015E2B8B
:108990000001ECE3396A400E386E1C0E376E8B0E08
:1089A000366E68C133F067C132F013EC08F004ECA6
:1089B00007F035C018F434C017F433C016F432C0D1
:1089C00015F4120001016A6B696B686B676B5E6B73
:1089D0000A0E01015E5D000119E2040EEAEC02F0EC
:1089E0000C6E25C00DF00C50010169270D506A2353
:1089F0000F0EEAEC02F00C6E25C00DF00C5067274C
:108A00000D50682301015E2B0001E2E30101695171
:108A1000675D0401196F01016A51685904011A6FF9
:108A20001AC420F019C41FF01A6A050E196EEEEC74
:108A300003F0196F12C01AF4396A400E386E1C0E1A
:108A4000376E8B0E366E68C133F067C132F013ECAF
:108A500008F004EC07F035C018F434C017F433C044
:108A600016F432C015F400EE80F0020E016E086AB2
:108A70001AC41AF019C419F09EEC00F0EF6A00EE67
:108A800086F0020E016E18C427F017C426F016C433
:108A900025F015C424F0DDEC00F0EF6A00011200AF
:108AA000949A8B8A010156510001E8B81CD0800EBF
:108AB000026E400E096E226A3DC421F0066A056A04
:108AC000200E016E110EF76E660EF66E0900F5505F
:108AD00003E0A5EC01F0FAD70D0EA5EC01F00A0EAB
:108AE000A5EC01F03BD0800E026E400E096E226AAA
:108AF0003DC421F0066A056A200E016EB50EA5EC94
:108B000001F0620EA5EC01F0060EA5EC01F0570E87
:108B1000A5EC01F0080EA5EC01F0000EA5EC01F0AB
:108B2000010EA5EC01F0000EA5EC01F0000EA5EC85
:108B300001F0000EA5EC01F0500EA5EC01F04F0E77
:108B4000A5EC01F0540EA5EC01F0530EA5EC01F0DC
:108B5000AC0EA5EC01F0850EA5EC01F0A20ED36ED3
:108B6000D288C290719E020E166E710E63EC03F0F5
:108B7000D298D20ED36EC280718E949A8B9A0101D4
:108B800056510001E8B81CD0800E026E400E096EEE
:108B9000226A3DC421F0066A056A200E016E110E9C
:108BA000F76E740EF66E0900F55003E0A5EC01F0C7
:108BB000FAD70D0EA5EC01F00A0EA5EC01F03BD0A2
:108BC000800E026E400E096E226A3DC421F0066AD4
:108BD000056A200E016EB50EA5EC01F0620EA5EC43
:108BE00001F0060EA5EC01F0570EA5EC01F0080E01
:108BF000A5EC01F0000EA5EC01F0010EA5EC01F0D2
:108C0000000EA5EC01F0000EA5EC01F0000EA5ECA5
:108C100001F0200EA5EC01F04E0EA5EC01F0550E72
:108C2000A5EC01F0520EA5EC01F07B0EA5EC01F0D5
:108C3000C30EA5EC01F0130E166E880E63EC03F064
:108C4000096A010E026E18EC02F0D8A029D70101C2
:108C5000606F000125D73DC448F002EE49F0240EB4
:108C6000EE6E470EEE6EEF6A800E026E800E096E9B
:108C7000226A3DC421F00B0E066EB80E056E63EC41
:108C800001F0D8A04BD02408FAE163EC01F0D8A0A1
:108C900045D00101606F020E5E6F510E01015E5DF5
:108CA00000011BE2800E026E800E096E226A3DC436
:108CB00021F081EC01F00101606F02EE49F05E519C
:108CC000E926000EEA2260C1EFFF0D0E605D000193
:108CD00004E001015E2B0001E0E30D6A01015E2961
:108CE0000C6ED8B40D2A0C50490FE96E020E0D20FF
:108CF000EA6EEF6A5F6B01015F515E5D00010EE39A
:108D000002EE49F001015F51E926000EEA22EF5020
:108D100046EC02F001015F2B0001EDE3030E096E4A
:108D2000E80E026E18EC02F0D8A095D70101606F32
:108D3000550E605D010ED8A4000E3B6E750E605D91
:108D4000010ED8A4000E3B12000109E004013D2BE6
:108D5000016A3D51A0EC00F00D0E46EC02F0440E0D
:108D60000101605D010ED8A4000E3B6E640E605DD3
:108D7000010ED8A4000E3B12000109E004013D07DA
:108D8000016A3D51A0EC00F00D0E46EC02F0530ECE
:108D90000101605D010ED8A4000E3B6E730E605D94
:108DA000010ED8A4000E3B1200011AE0AA6A3B0E85
:108DB000A96E04013D51DBEC02F00D0E46EC02F011
:108DC0001E0EF76E4C0EF66E3EEC02F0016A3D513F
:108DD000A0EC00F00D0E46EC02F00001EBEF39F0D4
:108DE000450E0101605D010ED8A4000E3B6E650EBC
:108DF000605D010ED8A4000E3B12000116E048C0D1
:108E00003DF40D0E46EC02F01E0EF76E540EF66E9B
:108E10003EEC02F0016A04013D51A0EC00F00D0EA1
:108E200046EC02F00001EBEF39F017D701015531A4
:108E30000001D8A0120002EE49F01E0EF76E700E6F
:108E4000F66E89EC04F0020E016E086A1A6A050ECD
:108E5000196EA3EC00F02E0EEE6E020E016E010EE6
:108E6000086E380EA1EC00F00D0EEE6EEE6A18ECF6
:108E700024F000EEE9F01E0EF76E7A0EF66E89EC25
:108E800004F0EE6A600E4D6E2DEC39F000EEE9F064
:108E900010EE4EF0080EE75204E0E6CFEEFFE82EAB
:108EA000FAD7EF6A610E4D6E2DEC39F0030E4A6E63
:108EB0006BEC23F0F00E4A6E6BEC23F001015E6B5D
:108EC000640E01015E5D000112E202EE49F0010153
:108ED0005E51E926000EEA22EF504A6E4A52000126
:108EE00006E06BEC23F001015E2B0001E9E329ECC5
:108EF00024F001015B97010E166EF40E63EC03F093
:108F000000011200080E0301DF6FA10EDE6F790E63
:108F1000DD6FDC6BC8C335F0C7C334F0C6C333F0B4
:108F2000C5C332F0396A386AA80E376E860E366EBF
:108F3000F2EC05F03B6EC8C335F0C7C334F0C6C3CE
:108F400033F0C5C332F0396A386AC80E376E840E02
:108F5000366E2EEC06F03B16000109E0080E030108
:108F6000DF6F9B0EDE6F370EDD6F700EDC6F000162
:108F7000C4C335F0C3C334F0C2C333F0C1C332F04D
:108F8000CD0E396ECC0E386E8B0E376E840E366E6B
:108F9000F2EC05F03B6EC4C335F0C3C334F0C2C37A
:108FA00033F0C1C332F08F0E396EC20E386E650ECB
:108FB000376E810E366E2EEC06F03B16C8C335F0C8
:108FC000C7C334F0C6C333F0C5C332F08F0E396E59
:108FD000420E386E980E376E850E366EF2EC05F046
:108FE0003B16C8C335F0C7C334F0C6C333F0C5C39E
:108FF00032F0140E396EAE0E386ED30E376E830E0D
:10900000366E2EEC06F03B1609E0080E0301DF6F0A
:10901000AD0EDE6F380EDD6FD00EDC6F0001C4C305
:1090200035F0C3C334F0C2C333F0C1C332F03D0ED8
:10903000396E0A0E386E6B0E376E830E366EF2EC9A
:1090400005F03B6EC4C335F0C3C334F0C2C333F084
:10905000C1C332F0660E396E386E3C0E376E840E28
:10906000366E2EEC06F03B16C8C335F0C7C334F09D
:10907000C6C333F0C5C332F0EC0E396E510E386EF4
:109080007E0E376E850E366EF2EC05F03B16C8C3C9
:1090900035F0C7C334F0C6C333F0C5C332F0290E70
:1090A000396E9C0E386E190E376E860E366E2EECAB
:1090B00006F03B1609E0080E0301DF6F9F0EDE6F1E
:1090C000560EDD6F200EDC6F0001C4C335F0C3C344
:1090D00034F0C2C333F0C1C332F0480E396EE10E32
:1090E000386E0E0E376E830E366EF2EC05F03B6E68
:1090F000C4C335F0C3C334F0C2C333F0C1C332F0CC
:10910000C30E396EF50E386E560E376E840E366EFF
:109110002EEC06F03B16C8C335F0C7C334F0C6C307
:1091200033F0C5C332F09A0E396E190E386E120E36
:10913000376E850E366EF2EC05F03B16C8C335F07F
:10914000C7C334F0C6C333F0C5C332F08F0E396ED7
:10915000C20E386E060E376E860E366E2EEC06F098
:109160003B1608E0080E0301DF6F9F0EDE6F080E4E
:10917000DD6FDC6B0001C4C335F0C3C334F0C2C380
:1091800033F0C1C332F0850E396EEB0E386E290E06
:10919000376E840E366EF2EC05F03B6EC4C335F0CC
:1091A000C3C334F0C2C333F0C1C332F0E10E396E31
:1091B0007A0E386E4E0E376E840E366E2EEC06F03A
:1091C0003B16C8C335F0C7C334F0C6C333F0C5C3BC
:1091D00032F00A0E396ED70E386E300E376E850EAD
:1091E000366EF2EC05F03B16C8C335F0C7C334F059
:1091F000C6C333F0C5C332F0E10E396E7A0E386E55
:109200006D0E376E850E366E2EEC06F03B1608E0BE
:10921000080E0301DF6FA10EDE6F790EDD6FDC6BD0
:109220000001C4C335F0C3C334F0C2C333F0C1C3BB
:1092300032F0710E396E3D0E386E420E376E810E71
:10924000366EF2EC05F03B6EC4C335F0C3C334F0A8
:10925000C2C333F0C1C332F0290E396E5C0E386ED2
:10926000230E376E830E366E2EEC06F03B16C8C307
:1092700035F0C7C334F0C6C333F0C5C332F0D70EE0
:10928000396EA30E386E420E376E850E366EF2ECD6
:1092900005F03B16C8C335F0C7C334F0C6C333F07E
:1092A000C5C332F0CD0E396E4C0E386E520E376E8D
:1092B000850E366E2EEC06F03B1609E0080E030113
:1092C000DF6FAC0EDE6F890EDD6F080EDC6F000104
:1092D000C4C335F0C3C334F0C2C333F0C1C332F0EA
:1092E000F60E396E280E386EDA0E376E840E366E34
:1092F000F2EC05F03B6EC4C335F0C3C334F0C2C317
:1093000033F0C1C332F0520E396EB80E386E810E92
:10931000376E840E366E2EEC06F03B16C8C335F061
:10932000C7C334F0C6C333F0C5C332F0B80E396ECC
:109330009E0E386E210E376E860E366EF2EC05F0FC
:109340003B16C8C335F0C7C334F0C6C333F0C5C33A
:1093500032F0710E396EFD0E386E330E376E860E9A
:10936000366E2EEC06F03B1609E0080E0301DF6FA7
:109370009E0EDE6F0A0EDD6F180EDC6F0001C4C397
:1093800035F0C3C334F0C2C333F0C1C332F0140E9E
:10939000396EAE0E386EC80E376E840E366EF2EC35
:1093A00005F03B6EC4C335F0C3C334F0C2C333F021
:1093B000C1C332F05C0E396E8F0E386E8A0E376E76
:1093C000820E366E2EEC06F03B16C8C335F0C7C3CE
:1093D00034F0C6C333F0C5C332F09A0E396E990E1D
:1093E000386E530E376E850E366EF2EC05F03B1676
:1093F000C8C335F0C7C334F0C6C333F0C5C332F0B9
:10940000B80E396E9E0E386E210E376E860E366E91
:109410002EEC06F03B1609E0080E0301DF6FA70EE5
:10942000DE6F310EDD6FD80EDC6F0001C4C335F086
:10943000C3C334F0C2C333F0C1C332F0EC0E396E93
:10944000510E386EA80E376E820E366EF2EC05F0B5
:109450003B6EC4C335F0C3C334F0C2C333F0C1C3E1
:1094600032F05C0E396E8F0E386E420E376E810E02
:10947000366E2EEC06F03B16C8C335F0C7C334F089
:10948000C6C333F0C5C332F0F60E396EA80E386E7F
:109490003D0E376E850E366EF2EC05F03B16C8C3F6
:1094A00035F0C7C334F0C6C333F0C5C332F0396AF0
:1094B000386A160E376E860E366E2EEC06F03B16A8
:1094C00009E0080E0301DF6F9B0EDE6F370EDD6FC4
:1094D000700EDC6F0001C4C335F0C3C334F0C2C3E7
:1094E00033F0C1C332F01F0E396E850E386E040E94
:1094F000376E840E366EF2EC05F03B6EC4C335F069
:10950000C3C334F0C2C333F0C1C332F01F0E396E8F
:10951000850E386E1A0E376E840E366E2EEC06F0FF
:109520003B16C8C335F0C7C334F0C6C333F0C5C358
:1095300032F08F0E396E420E386E7A0E376E850E0F
:10954000366EF2EC05F03B16C8C335F0C7C334F0F5
:10955000C6C333F0C5C332F01F0E396EC50E386E68
:10956000010E376E860E366E2EEC06F03B1609E0C5
:10957000080E0301DF6F9E0EDE6FB90EDD6FE00E89
:10958000DC6F0001C4C335F0C3C334F0C2C333F091
:10959000C1C332F0520E396EB80E386ECF0E376E30
:1095A000840E366EF2EC05F03B6EC4C335F0C3C3D7
:1095B00034F0C2C333F0C1C332F0F60E396E280E58
:1095C000386E9A0E376E830E366E2EEC06F03B1612
:1095D000C8C335F0C7C334F0C6C333F0C5C332F0D7
:1095E0009A0E396E190E386E8E0E376E850E366EE7
:1095F000F2EC05F03B16C8C335F0C7C334F0C6C360
:1096000033F0C5C332F0396A386AD60E376E840E2D
:10961000366E2EEC06F03B1609E0080E0301DF6FF4
:10962000A30EDE6F740EDD6FD00EDC6F0001C4C3BD
:1096300035F0C3C334F0C2C333F0C1C332F0396A6A
:10964000386A376A820E366EF2EC05F03B6EC4C3A0
:1096500035F0C3C334F0C2C333F0C1C332F0B80E27
:10966000396E1E0E386E310E376E820E366E2EEC4F
:1096700006F03B16C8C335F0C7C334F0C6C333F099
:10968000C5C332F0330E396EB30E386EAB0E376E83
:10969000850E366EF2EC05F03B16C8C335F0C7C335
:1096A00034F0C6C333F0C5C332F09A0E396E990E4A
:1096B000386EA50E376E850E366E2EEC06F03B1614
:1096C00008E0080E0301DF6FA10EDE6F790EDD6F7B
:1096D000DC6B0001C4C335F0C3C334F0C2C333F044
:1096E000C1C332F09A0E396E990E386E790E376E0C
:1096F0007F0E366EF2EC05F03B6EC4C335F0C3C38B
:1097000034F0C2C333F0C1C332F0480E396EE10EFB
:10971000386E4A0E376E820E366E2EEC06F03B1611
:10972000C8C335F0C7C334F0C6C333F0C5C332F085
:109730001F0E396E850E386E8F0E376E850E366EA3
:10974000F2EC05F03B16C8C335F0C7C334F0C6C30E
:1097500033F0C5C332F05C0E396E8F0E386EF20EE8
:10976000376E840E366E2EEC06F03B1609E0080EBE
:109770000301DF6FA40EDE6FAD0EDD6F500EDC6FE8
:109780000001C4C335F0C3C334F0C2C333F0C1C356
:1097900032F00A0E396ED70E386E630E376E810EB8
:1097A000366EF2EC05F03B6EC4C335F0C3C334F043
:1097B000C2C333F0C1C332F0E10E396E7A0E386E97
:1097C0001C0E376E820E366E2EEC06F03B16C8C3AA
:1097D00035F0C7C334F0C6C333F0C5C332F0520E00
:1097E000396EB80E386EA50E376E850E366EF2ECF9
:1097F00005F03B16C8C335F0C7C334F0C6C333F019
:10980000C5C332F05C0E396E8F0E386E9A0E376E0D
:10981000850E366E2EEC06F03B1609E0080E0301AD
:10982000DF6FA40EDE6FAD0EDD6F500EDC6F00013A
:10983000300ED2EC02F00401056FD4EC02F0066F9A
:10984000D4EC02F0076FD4EC02F0086F0301DC5196
:109850000401055D10E10301DD510401065D0BE12A
:109860000301DE510401075D06E10301DF5104013C
:10987000085D000112E0AA6A300EA96E0301DC51F6
:10988000DBEC02F0DD51DBEC02F0DE51DBEC02F050
:10989000DF51DBEC02F0000101D81200010E0301E0
:1098A000876F886F080E896F00016DEC43F003012C
:1098B00089510C6E640E0C5C000102E101015A83B7
:1098C0000301DB6B020EDA6F01015A510001E8B2AD
:1098D00092D01F0E0301DF5D000114E311E14A0E77
:1098E0000301DE5D00010EE30BE1DD0E0301DD5D32
:1098F000000108E305E1400E0301DC5D000102E325
:10990000000E01D0010E3B6E010E0301DC5DB10EB5
:10991000DD59080EDE59190EDF59000102E2000E72
:1099200001D0010E3B1605E0040E0301DA6F020EB2
:10993000DB6F140E0301DF5D000114E311E1DC0EA7
:109940000301DE5D00010EE30BE1930E0301DD5D1B
:10995000000108E305E1800E0301DC5D000102E384
:10996000000E01D0010E3B6E010E0301DC5D7F0E87
:10997000DD59ED0EDE59100EDF59000102E2000E36
:1099800001D0010E3B1605E0060E0301DA6F030E4F
:10999000DB6F0A0E0301DF5D000114E311E16E0EBF
:1099A0000301DE5D00010EE30BE1490E0301DD5D05
:1099B000000108E305E1C00E0301DC5D000102E3E4
:1099C000000E01D0010E3B6E810E0301DC5DBF0E67
:1099D000DD59760EDE59080EDF59000102E2000E55
:1099E00001D0010E3B1605E00C0E0301DA6F050EE7
:1099F000DB6F000151D0400E0301DC5D720EDD59BA
:109A0000050EDE592A0EDF59000105E2030E03019F
:109A1000DA6F010EDB6FC00E0301DC5DEC0EDD5969
:109A20004F0EDE591C0EDF59000105E2040E030142
:109A3000DA6F020EDB6F400E0301DC5D5A0EDD595A
:109A40000A0EDE59150EDF59000105E2060E03016C
:109A5000DA6F030EDB6FC00E0301DC5DD90EDD593A
:109A60003E0EDE590E0EDF59000105E2080E03011D
:109A7000DA6F040EDB6F400E0301DC5DCE0EDD59A4
:109A80008C0EDE590A0EDF59000105E20C0E0301AF
:109A9000DA6F050EDB6F0001146A080E136E126A8E
:109AA000116A1C6A1B6A1A6ADAC319F029EC04F0FD
:109AB00014C008F413C007F412C006F411C005F472
:109AC000E3C335F0E2C334F0E1C333F0E0C332F076
:109AD00015EC08F035C039F034C038F033C037F039
:109AE00032C036F008C435F007C434F006C433F091
:109AF00005C432F015EC08F004EC07F035C0D5F3DE
:109B000034C0D4F333C0D3F332C0D2F3E3C314F080
:109B1000E2C313F0E1C312F0E0C311F01C6A1B6A48
:109B20001A6ADAC319F0A9EC03F014C0CDF313C01C
:109B3000CCF312C0CBF311C0CAF3DFC314F0DEC301
:109B400013F0DDC312F0DCC311F0CDC31CF0CCC3A5
:109B50001BF0CBC31AF0CAC319F0A9EC03F014C070
:109B600027F013C026F012C025F011C024F0240401
:109B700001015E6FDFC314F0DEC313F0DDC312F02A
:109B8000DCC311F0CDC31CF0CCC31BF0CBC31AF067
:109B9000CAC319F0A9EC03F031C008F430C007F4CF
:109BA0002FC006F42EC005F4CDC335F0CCC334F07D
:109BB000CBC333F0CAC332F015EC08F035C039F02E
:109BC00034C038F033C037F032C036F008C435F056
:109BD00007C434F006C433F005C432F015EC08F0C5
:109BE00004EC07F035C0D1F334C0D0F333C0CFF369
:109BF00032C0CEF3356A346A336A7F0E326ED1C317
:109C000039F0D0C338F0CFC337F0CEC336F076EC9E
:109C100006F035C0D1F334C0D0F333C0CFF332C037
:109C2000CEF3356A346A336A920E326ED1C339F09C
:109C3000D0C338F0CFC337F0CEC336F06AEC07F0AC
:109C4000B8EC07F00301D66F33C0D7F334C0D8F3B4
:109C500035C0D9F3D8C3F8F3D7C3F7F3D6C3F6F3B7
:109C6000080E876F110E886F400E896F040E8A6F81
:109C70008B6B5EC18CF3F8C38DF3F7C38EF3F6C321
:109C80008FF3000145EF43F00F13171A1C1E1E1D22
:109C90001B1815110D0906030100000204070B0F24
:109CA000719E0401A36BA26BA16BA06BA76BA66B4B
:109CB000A56BA46BC5EC02F0EE0E8FEC02F0AA0EC1
:109CC0008FEC02F073EC02F0596F73EC02F0586FF6
:109CD00073EC02F05B6F73EC02F05A6F73EC02F0FE
:109CE0005D6F73EC02F05C6F73EC02F05F6F73EC0E
:109CF00002F05E6F73EC02F0616F73EC02F0606F64
:109D000073EC02F0636F71EC02F0626FA2EC02F090
:109D1000C5EC02F0EE0E8FEC02F0B60E8FEC02F006
:109D200073EC02F0656F73EC02F0646F73EC02F099
:109D3000676F73EC02F0666F73EC02F07F6F73EC89
:109D400002F07E6F73EC02F0816F73EC02F0806FB3
:109D500073EC02F0836F71EC02F0826FA2EC02F000
:109D600000011200719E8BD8A7C487F4A6C486F4A4
:109D7000A5C485F4A4C484F4A3C48BF4A2C48AF457
:109D8000A1C489F4A0C488F4C80E62EC03F077D8AB
:109D9000A7C493F4A6C492F4A5C491F4A4C490F407
:109DA000A3C497F4A2C496F4A1C495F4A0C494F4F7
:109DB000C80E62EC03F063D804018451A425246E1C
:109DC0008551A521256E8651A621266E8751A72192
:109DD000276E90512424846F91512520856F9251D4
:109DE0002620866F93512720876F87C414F086C47E
:109DF00013F085C412F084C411F01C6A1B6A1A6A3D
:109E0000030E196EA9EC03F014C0A7F413C0A6F456
:109E100012C0A5F411C0A4F494518825246E955164
:109E20008921256E96518A21266E97518B21276EA6
:109E3000A0512424886FA1512520896FA25126208A
:109E40008A6FA35127208B6F8BC414F08AC413F040
:109E500089C412F088C411F01C6A1B6A1A6A030EC6
:109E6000196EA9EC03F014C0A3F413C0A2F412C03D
:109E7000A1F411C0A0F4000148D8718E1200C5EC05
:109E800002F0EE0E8FEC02F0F40E8FEC02F02E0ECC
:109E90008DEC02F0050E62EC03F0EE0E8FEC02F09A
:109EA000F60E8FEC02F073EC02F00401B16F71EC6E
:109EB00002F0B06FA2EC02F0B1C4A1F4B0C4A0F4FF
:109EC000C5EC02F0EE0E8FEC02F0F40E8FEC02F017
:109ED000340E8DEC02F0050E62EC03F0EE0E8FEC0A
:109EE00002F0F60E8FEC02F073EC02F0B26F73EC3E
:109EF00002F0B16F71EC02F0B06FA2EC02F0B2C4EC
:109F0000A5F4B1C4A4F40001120004016251A05DE3
:109F1000326E6351A159336E000E63BFFF0EA2591A
:109F2000346E000E63BFFF0EA359356E17EC08F0B8
:109F300035C027F034C026F033C025F032C024F0FD
:109F400061C433F060C432F00BEC08F027C039F084
:109F500026C038F025C037F024C036F06AEC07F090
:109F600035C066F134C065F133C064F132C063F1CD
:109F700066C1BBF465C1BAF464C1B9F40F0E010146
:109F8000635D02E23E84000E0401B86F81C433F0C9
:109F900080C432F00BEC08F035C027F034C026F056
:109FA00033C025F032C024F00B0E242402E33E829D
:109FB000FF0E0001246EBBC42BF0BAC42AF0B9C452
:109FC00029F0B8C428F083C433F082C432F00BEC1B
:109FD00008F02BC039F02AC038F029C037F028C06B
:109FE00036F076EC06F035C02BF034C02AF033C0E2
:109FF00029F032C028F027C035F026C034F025C043
:10A0000033F024C032F02BC039F02AC038F029C018
:10A0100037F028C036F004EC07F035C0BFF434C088
:10A02000BEF433C0BDF432C0BCF4BBC439F0BAC412
:10A0300038F0B9C437F0B8C436F0BFC435F0BEC488
:10A0400034F0BDC433F0BCC432F076EC06F035C059
:10A05000CFF434C0CEF433C0CDF432C0CCF4356A82
:10A06000346A336A820E326ECFC439F0CEC438F00F
:10A07000CDC437F0CCC436F076EC06F035C027F00E
:10A0800034C026F033C025F032C024F0396A386A73
:10A09000376A830E366E27C035F026C034F025C0EF
:10A0A00033F024C032F004EC07F0B8EC07F0040100
:10A0B000A86F33C0A9F434C0AAF435C0ABF4396A30
:10A0C000386A200E376E820E366EABC435F0AAC4E5
:10A0D00034F0A9C433F0A8C432F017EC08F004EC53
:10A0E00007F035C00FF534C00EF533C00DF532C0A2
:10A0F0000CF500EED3F0020E016E0FC527F00EC571
:10A1000026F00DC525F00CC524F0010EDDEC00F0A5
:10A11000EF6A396A386A7A0E376E8A0E366ECFC4A5
:10A1200035F0CEC434F0CDC433F0CCC432F074EC8E
:10A1300006F035C0D3F434C0D2F433C0D1F432C009
:10A14000D0F4D3C439F0D2C438F0D1C437F0D0C47D
:10A1500036F0D3C435F0D2C434F0D1C433F0D0C417
:10A1600032F06AEC07F035C027F034C026F033C077
:10A1700025F032C024F027C066F126C065F125C065
:10A1800064F10C0E245C02E23E84000E0101636F58
:10A1900067C433F066C432F00BEC08F066C139F0E6
:10A1A00065C138F064C137F063C136F06AEC07F07E
:10A1B00035C0BBF434C0BAF433C0B9F432C0B8F41B
:10A1C0005BC433F05AC432F00BEC08F0D3C439F05E
:10A1D000D2C438F0D1C437F0D0C436F06AEC07F0FE
:10A1E00035C0BFF434C0BEF433C0BDF432C0BCF4DB
:10A1F000BBC439F0BAC438F0B9C437F0B8C436F0CB
:10A20000BFC435F0BEC434F0BDC433F0BCC432F0BA
:10A2100076EC06F035C027F034C026F033C025F0C8
:10A2200032C024F027C0C3F426C0C2F425C0C1F454
:10A230000B0E245C02E23E84000E0401C06F59C480
:10A2400033F058C432F00BEC08F035C027F034C0BE
:10A2500026F033C025F032C024F0020E242402E39D
:10A260003E82FF0E0001246E27C039F026C038F070
:10A2700025C037F024C036F0C3C435F0C2C434F072
:10A28000C1C433F0C0C432F076EC06F035C027F01C
:10A2900034C026F033C025F032C024F0356A346A69
:10A2A000336A800E326E27C039F026C038F025C0E0
:10A2B00037F024C036F076EC06F035C027F034C015
:10A2C00026F033C025F032C024F027C0C7F426C0E2
:10A2D000C6F425C0C5F4020E245C02E23E84000EE2
:10A2E0000401C46F5DC433F05CC432F00BEC08F0C1
:10A2F000D3C439F0D2C438F0D1C437F0D0C436F06A
:10A300006AEC07F035C027F034C026F033C025F0E2
:10A3100032C024F027C0BBF426C0BAF425C0B9F47B
:10A320000D0E245C02E23E84000E0401B86F65C489
:10A3300033F064C432F00BEC08F066C139F065C14B
:10A3400038F064C137F063C136F06AEC07F035C00D
:10A3500027F034C026F033C025F032C024F027C0E7
:10A36000BFF426C0BEF425C0BDF4100E245C02E28A
:10A370003E84000E0401BC6FBBC427F0BAC426F0B3
:10A38000B9C425F0B8C424F027C039F026C038F08D
:10A3900025C037F024C036F0BFC435F0BEC434F059
:10A3A000BDC433F0BCC432F076EC06F035C027F003
:10A3B00034C026F033C025F032C024F0356A346A48
:10A3C000336A800E326E27C039F026C038F025C0BF
:10A3D00037F024C036F076EC06F035C027F034C0F4
:10A3E00026F033C025F032C024F027C0C3F426C0C5
:10A3F000C2F425C0C1F4020E245C02E23E84000EC9
:10A400000401C06F5FC433F05EC432F013EC08F097
:10A4100035C027F034C026F033C025F032C024F018
:10A42000C3C42BF0C2C42AF0C1C429F0C0C428F0B0
:10A43000356A346A336A8E0E326E2BC039F02AC008
:10A4400038F029C037F028C036F076EC06F035C079
:10A450002BF034C02AF033C029F032C028F027C0D6
:10A4600039F026C038F025C037F024C036F02BC0B4
:10A4700035F02AC034F029C033F028C032F06AEC3D
:10A4800007F035C027F034C026F033C025F032C0C5
:10A4900024F027C0CBF426C0CAF425C0C9F40F0E9F
:10A4A000245C02E23E84000E0401C86FA7C435F0AC
:10A4B000A6C434F0A5C433F0A4C432F017EC08F0FD
:10A4C000C7C439F0C6C438F0C5C437F0C4C436F0C8
:10A4D00074EC06F035C027F034C026F033C025F008
:10A4E00032C024F0356A500E346E430E336E8E0E39
:10A4F000326E27C039F026C038F025C037F024C0AE
:10A5000036F06AEC07F0B8EC07F0786F33C079F4F6
:10A5100034C07AF435C07BF47BC435F07AC434F0AF
:10A5200079C433F078C432F017EC08F0396A386A2D
:10A53000376A800E366E6AEC07F035C027F034C0FB
:10A5400026F033C025F032C024F027C035F026C0F5
:10A5500034F025C033F024C032F0CBC439F0CAC483
:10A5600038F0C9C437F0C8C436F004EC07F035C081
:10A57000D7F434C0D6F433C0D5F432C0D4F4D7C441
:10A5800066F1D6C465F1D5C464F1080ED45D02E26B
:10A590003E84000E0101636F66C139F065C138F079
:10A5A00064C137F063C136F066C135F065C134F07F
:10A5B00064C133F063C132F06AEC07F035C0BBF41C
:10A5C00034C0BAF433C0B9F432C0B8F4356AE00E1E
:10A5D000346E3D0E336E8A0E326EBBC439F0BAC48F
:10A5E00038F0B9C437F0B8C436F06AEC07F035C0BB
:10A5F00027F034C026F033C025F032C024F027C045
:10A60000BBF426C0BAF425C0B9F4100E245C02E2F3
:10A610003E84000E0401B86F356AE80E346EE50E14
:10A62000336E8B0E326ED7C439F0D6C438F0D5C431
:10A6300037F0D4C436F06AEC07F035C027F034C0E8
:10A6400026F033C025F032C024F027C0BFF426C066
:10A65000BEF425C0BDF4100E245C02E23E84000E60
:10A660000401BC6FD7C427F0D6C426F0D5C425F0AA
:10A67000D4C424F0BBC42BF0BAC42AF0B9C429F066
:10A68000B8C428F02BC039F02AC038F029C037F000
:10A6900028C036F0BFC435F0BEC434F0BDC433F0BA
:10A6A000BCC432F076EC06F035C02BF034C02AF092
:10A6B00033C029F032C028F0356AF00E346E6C0ECB
:10A6C000336E8A0E326E2BC039F02AC038F029C0A2
:10A6D00037F028C036F076EC06F035C02BF034C0E9
:10A6E0002AF033C029F032C028F0040E285E02E2BE
:10A6F0003E84286A000127C039F026C038F025C002
:10A7000037F024C036F02BC035F02AC034F029C011
:10A7100033F028C032F076EC06F0B8EC07F0040114
:10A72000AC6F33C0ADF434C0AEF435C0AFF4396AA9
:10A73000386A480E376E850E366EAFC435F0AEC43B
:10A7400034F0ADC433F0ACC432F017EC08F004ECD4
:10A7500007F035C027F034C026F033C025F032C0F2
:10A7600024F09A0E356E990E346E550E336E830EAC
:10A77000326E27C039F026C038F025C037F024C02B
:10A7800036F076EC06F035C0D7F434C0D6F433C0DA
:10A79000D5F432C0D4F400EEC8F0020E016ED7C476
:10A7A00027F0D6C426F0D5C425F0D4C424F0010E79
:10A7B000DDEC00F0EF6A00011200B50E0301876FB7
:10A7C000620E886F060E896F240E8A6F8B6F8C6BFA
:10A7D0008D698E69080E8F6F030E906F916B926B6F
:10A7E000936B946B100E956F270E966F976B986B0B
:10A7F000050E996F9A6BFA0E9B6F9C6B9D6F9E6B0B
:10A80000640E9F6FA06B2C0EA16F010EA26FA36B45
:10A81000A46BA56BA66BA76BA86BA96BAA6BAB6BA4
:10A82000AC6BAD6BAE6BAF6BB06B160EB16FDC0E7D
:10A83000B26FB16BB26B020E01015E6F2A0E0101A5
:10A840005E5D00011AE20301B1510E6E03EE87F066
:10A8500001015E51EB50106E0E240C6E0CC0B1F372
:10A860000301B2510E6EB151106E0E240C6E0CC06D
:10A87000B2F301015E2B0001E1E301015E6B2C0EDE
:10A8800001015E5D00010BE203EE87F001015E5104
:10A89000EB5013EC02F001015E2B0001F0E389C3E1
:10A8A0000CF00CC08DF38AC30CF00CC08EF3B50E07
:10A8B0000301876F620E886F050E896F010E8A6F24
:10A8C000020E8B6F8C6B8F6B906B020E01015E6FB3
:10A8D000080E01015E5D00011AE203018F510E6E48
:10A8E00003EE87F001015E51EB50106E0E240C6EEA
:10A8F0000CC08FF3030190510E6E8F51106E0E2419
:10A900000C6E0CC090F301015E2B0001E1E30B0E15
:10A91000096EB80E026EEDEC01F037E30101606FD5
:10A92000030187510C6E010160510C5C00010BE0CA
:10A930000B0E096EB80E026EEDEC01F026E301017C
:10A94000606F0001EDD7010E01015E6F080E01017D
:10A950005E5D000116E20B0E096EB80E026EEDECA4
:10A9600001F013E30101606F03EE87F05E51EB50DD
:10A970000C6E60510C5C000108E101015E2B0001CE
:10A98000E5E301015A970001120001015A87000115
:10A99000120094988B88100E0F01406FDFC3EBF309
:10A9A000DEC3EAF3DDC3E9F3DCC3E8F30301EC51F2
:10A9B000E425DC6FED51E521DD6F000EEDBFFF0EEC
:10A9C000E621DE6F000EEDBFFF0EE721DF6F000115
:10A9D0004EEC4CF0D4EC20F001015631000107E3BD
:10A9E0003AEC1EF0030E166EE80E63EC03F0010164
:10A9F00056350001D8B013D832EC20F0EBC3DFF3AA
:10AA0000EAC3DEF3E9C3DDF3E8C3DCF34EEC4CF05C
:10AA10002EEC21F077EC20F094988B981200040132
:10AA2000396B02EE49F011EE9DF0550EE75204E04D
:10AA3000E6CFEEFFE82EFAD7EF6A01015F6B000167
:10AA40005AEC21F003015451C96F01EE0DF0EF6A89
:10AA500001EE1DF0EF6A01EE2DF0EF6A03EE4EF00D
:10AA6000EF6A01015F6B00018BEC21F002EE49F00F
:10AA700001015F51E926000EEA22EFCF0CF00CC075
:10AA80000DF10F6A5F290E6ED8B40F2A0E50490FD0
:10AA9000E96E020E0F20EA6EEFCF0CF00CC00EF143
:10AAA0003A0E0F6F0F6A020E5F250E6ED8B00F2A96
:10AAB0000E50490FE96E020E0F20EA6EEFCF0CF038
:10AAC0000CC010F10F6A030E5F250E6ED8B00F2A6E
:10AAD0000E50490FE96E020E0F20EA6EEFCF0CF018
:10AAE0000CC011F13A0E126F0F6A040E5F250E6E44
:10AAF000D8B00F2A0E50490FE96E020E0F20EA6EF1
:10AB0000EFCF0CF00CC013F10F6A050E5F250E6E2F
:10AB1000D8B00F2A0E50490FE96E020E0F20EA6ED0
:10AB2000EFCF0CF00CC014F1156B5F6B00015EEC05
:10AB300021F001EE1DF013EE54F0080EE6CFEEFF0B
:10AB4000E82EFCD7EF6A01015F6B00015DEC21F09C
:10AB500003EE54F0EECFF3FFEFCFF4FFF350530AC0
:10AB6000F4101AE103EE54F02D0EEE6E11EE1DF00E
:10AB70000F0EE75204E0E6CFEEFFE82EFAD7EF6AB9
:10AB800001EE1DF013EE54F0320EE75204E0E6CF72
:10AB9000EEFFE82EFAD7EF6A01015F6B00015CEC73
:10ABA00021F001EE2DF013EE54F0090EE6CFEEFF8A
:10ABB000E82EFCD7EF6A01015F6B00015BEC21F02E
:10ABC00003EE54F0EECFF3FFEFCFF4FFF350570A4C
:10ABD000F4101AE103EE54F02D0EEE6E11EE2DF08E
:10ABE0000F0EE75204E0E6CFEEFFE82EFAD7EF6A49
:10ABF00001EE2DF013EE54F0320EE75204E0E6CFF2
:10AC0000EEFFE82EFAD7EF6A01015F6B000159EC05
:10AC100021F003EE4EF013EE54F0320EE75204E052
:10AC2000E6CFEEFFE82EFAD7EF6A03EE4EF004EC23
:10AC300000F004013B6F01015F6B000157EC21F054
:10AC4000040E04013B5D000114E301EE3DF013EE40
:10AC500054F0320EE75204E0E6CFEEFFE82EFAD7CA
:10AC6000EF6A01EE3DF004EC00F00401336F1AC00E
:10AC700034F401015E6B060E01015E5D00010EE21F
:10AC800000EE4EF001015E51EB500C6E200E0C5C9C
:10AC9000000104E001015E2B0001EDE300EEE9F0AC
:10ACA000240EEE6EEE6EEE6EEE6E10EE4EF00101C4
:10ACB0005E51E6CFEEFFE82EFCD7EF6A00EEE9F03A
:10ACC000EE50FEE1ED522F0EEE6E410EEE6E4D0E89
:10ACD000EE6E2C0EEE6E13EE4EF0050EE75204E013
:10ACE000E6CFEEFFE82EFAD72C0EEE6E11EE0DF049
:10ACF0000F0EE75204E0E6CFEEFFE82EFAD72C0E57
:10AD0000EE6E11EE1DF00F0EE75204E0E6CFEEFFFF
:10AD1000E82EFAD72C0EEE6E11EE2DF00F0EE75244
:10AD200004E0E6CFEEFFE82EFAD7EF6A5D310001CE
:10AD3000D8B088D000EEE9F0EE50FEE1ED522C0ED6
:10AD4000EE6E11EE3DF00F0EE75204E0E6CFEEFF9F
:10AD5000E82EFAD7EF6A010156510001E8AA17D090
:10AD6000B2EC4EF000EEE9F0EE50FEE1ED522C0EAA
:10AD7000EE6E020E016ED7C427F0D6C426F0D5C4FD
:10AD800025F0D4C424F0010EDDEC00F0EF6A0101DF
:10AD900057510001E8A617D0C3EC43F000EEE9F0EC
:10ADA000EE50FEE1ED522C0EEE6E020E016E1EC450
:10ADB00027F01DC426F01CC425F01BC424F0010E8E
:10ADC000DDEC00F0EF6A010157510001E8A414D056
:10ADD00000EEE9F0EE50FEE1ED522C0EEE6E020EAA
:10ADE000016E14C427F013C426F012C425F011C458
:10ADF00024F0DDEC00F0EF6A010156510001E8A6F5
:10AE000021D0E2EC44F000EEE9F0EE50FEE1ED522C
:10AE10002C0EEE6E020E016E18C427F017C426F039
:10AE200016C425F015C424F0DDEC00F02C0EEE6EF7
:10AE3000020E016E086A1AC41AF019C419F09EECC9
:10AE400000F0EF6A0401576B00EEE9F0E86AEE5299
:10AE500002E0E83EFCD70B6E040E01015F6F0101BA
:10AE60005F510B5C00010CE300EEE9F001015F5162
:10AE7000EB500C6E0401571B01015F2B0001EFE347
:10AE800000EEE9F0EE50FEE1ED522A0EEE6E020EFB
:10AE9000016E086E0401575189EC00F00D0EEE6E44
:10AEA0000A0EEE6EEF6A0001939A8A8A23EC20F074
:10AEB0006DEC20F0640E62EC03F001015E6B0001AA
:10AEC00000EEE9F001015E51EB500C6E000E0C52E9
:10AED000D8A4010E3B6E960E5E5D010ED8B0000E3A
:10AEE0003B1600010DE000EEE9F001015E51EB5070
:10AEF0000401306F000109D801015E2B0001DFD78A
:10AF0000640E62EC03F077EF20F0939A8A9A0CC4F7
:10AF100012F004010B5170EC03F0010E0101606F9F
:10AF2000010160510301F45D000110E3040130B13F
:10AF3000818A30A1819A0CC412F00B5170EC03F09D
:10AF4000D89030330101602B0001EAE3939A8A8A9A
:10AF50000EC412F004010D5170EC03F00001120058
:08AF60000400FED70400FED737
:020000040030CA
:03000100D80E3BDB
:020005003D803C
:0600080008C00FE00F40EC
:0200000400F00A
:100000004F4D334243200B4243504C353500574946
:1000100044453120010000000000000057494445DC
:10002000322002778600280F2F4F028A0302C06910
:100030000079A1086407F82401B0045414C06B9E31
:10004000085203640007026A293F3E3C38302021F1
:1000500023272F475501310611150902140B1004EF
:100060001E0D1207050F161B0A08030C180E191D8A
:10007000134243545241434B20762E5C5A202D208C
:10008000556261743D205C75562C2054313D205CD6
:0400900054430D00C8
:00000001FF
